:100000000C9403050C942B050C942B050C942B05D8
:100010000C942B050C942B050C942B050C942B05A0
:100020000C942B050C942B050C94EA190C945C1A77
:100030000C942B050C942B050C942B050C942B0580
:100040000C942B050C942B050C942B050C942B0570
:100050000C942B050C942B050C942B050C941D1D56
:100060000C942B050C942B050C942B050C942B0550
:100070000C942B050C942B050C942B050C942B0540
:100080000C942B050C942B050C942B050C942B0530
:100090000C942B050C942B050C942B050C942B0520
:1000A0000C942B050C942B050C942B05810A930AB8
:1000B000F50AC80AED0A120B400ACC23D723E22323
:1000C000E923F72302240F241A242324232477244A
:1000D0007F248824F0F89C8E8783878E9CF8F0001C
:1000E00000FEFF0303030303070EFCF80000FEFFFE
:1000F0000303030303070EFCF80000FFFF000000EA
:1001000000000000FFFF0000FEFF8383838383C79E
:10011000EE7C380000F8FC0E07030303070EFCF822
:1001200000003F7FE0C08080C0E07F3FFFFF010113
:100130000101010101FFFF0000FFFF0C0C0C0C1C72
:100140003E77E3C100007FFFC0C0C0C0C0E0703F89
:100150001F00001F3F70E0C0C0C0E0703F1F0000E4
:100160007FFFC1C1C1C1C1E3773E1C00001F3F70CA
:10017000E0C0C0C0E0703F1F000000000001FFFFB2
:1001800001000000D5F08D14A1C881CFD9F1AF20B6
:10019000005265616C6C793F20413D7920423D6E93
:1001A000006E6577207265636F7264210067616D10
:1001B00065206F76657220617420006368656174E4
:1001C0002100191C1C1C1C19131307070707131304
:1001D00019F763B75F5B4140415B5F58414041584D
:1001E0005F5B4140415B5FAF47EF8055803E7F41A1
:1001F0006F6F717F3E0003017F0103007F41633E0B
:10020000807F800303020100010001000100010062
:10021000010001000100010001020303AA55AA55D3
:10022000AA55AA55080800000054007C0038003880
:10023000007C00540000000E0058007000300038B0
:100240000078005800100000004C005E0057025774
:100250000077002200000006006C00380018001C27
:10026000007E044E000C0004001E007C00380038A4
:10027000007C001E00040010009800CB007F007F6F
:1002800000CB00980010009200D6007C007E007E1B
:10029000007C00D60092000C0078003E047F047FB2
:1002A000003E0078000C0007008C00FC003F003F7F
:1002B00000FC008C0018000F005C00F800BC007F00
:1002C00004DF008E000C0033009A00FF047F047FDF
:1002D00000FF009A0033FFFFFFFFFFFFFFFFFF83D8
:1002E000C1E1E1C183FFFF83F9FDFDF983FFFFFF5A
:1002F000FFAA55FFFFFFF7EFF7EFF7EFF7EFFFFF6D
:10030000FFFAF5EBF7EFFFFFFFBF5FAFD7EFF7EBBC
:10031000F5FAFDFFFFFFF7EFD7AF5FFFFFFFFFFF2E
:10032000FFAA55EFF7EFF7EFF7AF57EFF7EFF7EF5C
:10033000F7AA55FFFFFFF7EFF7EAF5EFF7EFF7EF53
:10034000F7AA55EFF7EF080B0002020201000904BB
:100350000000010202000005240010010524010133
:10036000010424020605240600010705810310008C
:100370004009040100020A000000070502024000D3
:100380000007058302400000040309041201000273
:10039000EF02014041233680000101020301417256
:1003A0006475696E6F204C4C430041726475626FD6
:1003B00079001010FFFF3F3F8793B9E5E5B99387B8
:1003C0003F3FFFFFFFFFFF8E96B096BFBF96B096F0
:1003D0008EFFFFFFFFFF3FBF87838199998183874E
:1003E000BF3FFFFFFFFFFF8EA680A08080A080A6FA
:1003F0008EFFFFFFFFFFFFE3C91D73E7E7731DC912
:10040000E3FFFFFFFFFFFB91A4B495BFBF95B4A42A
:1004100091FBFFFFFFFFFFE3C9193307073319C93A
:10042000E3FFFFFFFFFFFB95A484A48E8EA484A4AA
:1004300095FBFFFF0102040810204080000000002F
:10044000003E5B4F5B3E3E6B4F6B3E1C3E7C3E1C5A
:10045000183C7E3C181C577D571C1C5E7F5E1C00A0
:10046000183C1800FFE7C3E7FF0018241800FFE757
:10047000DBE7FF30483A060E2629792926407F051A
:100480000507407F05253F5A3CE73C5A7F3E1C1C30
:1004900008081C1C3E7F14227F22145F5F005F5FF0
:1004A00006097F017F006689956A606060606094DC
:1004B000A2FFA29408047E040810207E20100808E1
:1004C0002A1C08081C2A08081E101010100C1E0CEC
:1004D0001E0C30383E3830060E3E0E06000000007E
:1004E0000000005F00000007000700147F147F1465
:1004F000242A7F2A122313086462364956205000AA
:1005000008070300001C2241000041221C002A1C95
:100510007F1C2A08083E0808008070300008080880
:100520000808000060600020100804023E514945A0
:100530003E00427F400072494949462141494D33BE
:100540001814127F1027454545393C4A4949314125
:10055000211109073649494936464949291E0000F3
:100560001400000040340000000814224114141448
:100570001414004122140802015909063E415D5934
:100580004E7C1211127C7F494949363E414141223D
:100590007F4141413E7F494949417F090909013E67
:1005A000414151737F0808087F00417F410020408E
:1005B000413F017F081422417F404040407F021CA0
:1005C000027F7F0408107F3E4141413E7F090909B7
:1005D000063E4151215E7F09192946264949493283
:1005E00003017F01033F4040403F1F2040201F3F49
:1005F0004038403F631408146303047804036159CE
:10060000494D43007F41414102040810200041410F
:10061000417F0402010204404040404000030708BB
:100620000020545478407F284444383844444428B7
:10063000384444287F385454541800087E0902185E
:10064000A4A49C787F0804047800447D40002040E6
:10065000403D007F1028440000417F40007C04782A
:1006600004787C080404783844444438FC18242472
:100670001818242418FC7C080404084854545424F2
:1006800004043F44243C4040207C1C2040201C3C6F
:100690004030403C44281028444C9090907C446466
:1006A000544C4400083641000000770000004136F9
:1006B000080002010204023C2623263C1EA1A1617F
:1006C000123A4040207A38545455592155557941B1
:1006D0002154547841215554784020545579400C88
:1006E0001E52721239555555593954545459395569
:1006F0005454580000457C410002457D42000145AC
:100700007C40F0292429F0F0282528F07C54554518
:10071000002054547C547C0A097F493249494932AB
:100720003248484832324A4848303A4141217A3AC0
:1007300042402078009DA0A07D39444444393D408A
:1007400040403D3C24FF2424487E4943662B2FFC37
:100750002F2BFF0929F620C0887E090320545479E5
:10076000410000447D413048484A32384040227AB6
:10077000007A0A0A727D0D19317D2629292F282633
:100780002929292630484D4020380808080808083B
:100790000808382F10C8ACBA2F102834FA00007B94
:1007A000000008142A142222142A1408950022009A
:1007B00095AA005500AAAA55AA55AA000000FF0054
:1007C000101010FF00141414FF001010FF00FF1091
:1007D00010F010F0141414FC001414F700FF0000C3
:1007E000FF00FF1414F404FC141417101F10101F42
:1007F000101F1414141F00101010F0000000001F30
:10080000101010101F10101010F010000000FF103A
:100810001010101010101010FF10000000FF140036
:1008200000FF00FF00001F10170000FC04F4141468
:100830001710171414F404F40000FF00F714141434
:1008400014141414F700F7141414171410101F10B4
:100850001F141414F4141010F010F000001F101FD7
:100860000000001F14000000FC140000F010F01045
:1008700010FF10FF141414FF141010101F000000BC
:1008800000F010FFFFFFFFFFF0F0F0F0F0FFFFFFC0
:100890000000000000FFFF0F0F0F0F0F3844443817
:1008A000447C2A2A3E147E02020606027E027E0252
:1008B00063554941633844443C04407E201E200671
:1008C000027E020299A5E7A5991C2A492A1C4C72AE
:1008D00001724C304A4D4D303048784830BC625A35
:1008E000463D3E494949007E0101017E2A2A2A2AC5
:1008F0002A44445F444440514A444040444A5140A1
:100900000000FF0103E080FF000008086B6B083661
:1009100012362436060F090F0600001818000000D2
:100920001010003040FF0101001F01011E00191DC1
:100930001712003C3C3C3C0000000000FFC399E55E
:10094000E599C3FFFFC199F3F399C1FFFFFFFBF9DD
:10095000FBEF87FFFFFBF9FBFF97A7FFFFBB93C7E9
:10096000C793BBFFFFFFFF81C3E7FFFFFFC399B53D
:10097000AD99C3FFFFE783818183E7FFFFE78B8D9D
:100980008D8BE7FFFFE783B1B183E7FFFF9981819B
:10099000818199FFFF99858D8D8599FFFF99A1B17F
:1009A000B1A199FFFF8F838181838FFFFF8F838D9B
:1009B0008D838FFFFF8FB3B1B1B38FFFFF9381831F
:1009C000838193FFFF938D8B8B8D93FFFF93A1B357
:1009D000B3A193FFFFF181838381F1FFFFF18D8B41
:1009E0008B8DF1FFFFF181B3B381F1FFFFEB8181CB
:1009F0008181EBFFFFEB858D8D85EBFFFFEB91B1E7
:100A0000B191EBFFC12E11241FBECFEFDAE0DEBFA4
:100A1000CDBF11E0A0E0B1E0EAEBF7E602C005903F
:100A20000D92AE39B107D9F729E0AEE9B1E001C0C6
:100A30001D92AD30B207E1F715E0C3E0D5E004C088
:100A40002197FE010E94F830C230D107C9F70E94F9
:100A500066260C94DB330C9400008F929F92AF9229
:100A6000BF92CF92DF92EF920F931F93CF93DF93BA
:100A7000FB016A01EB0183E0D695C7958A95E1F702
:100A8000CB01880F991F880F991F65E070E00E94C5
:100A9000D03042E0460FCF0163E070E00E94D030DA
:100AA000CF0104964801590154E0E52E0AE02C2FAD
:100AB000880F0E941622DF91CF911F910F91EF9026
:100AC000DF90CF90BF90AF909F908F9008958F92BE
:100AD0009F92AF92BF92CF92DF92EF920F931F93AC
:100AE000FB016A0159019B0183E0369527958A95A0
:100AF000E1F7CB01880F991F880F991F65E070E01F
:100B00000E94D030462FCF0163E070E00E94D030C9
:100B10008E2F880F480154E0E52E07E08D5F0E947C
:100B200016221F910F91EF90DF90CF90BF90AF9062
:100B30009F908F9008958F929F92AF92BF92CF9285
:100B4000DF92EF920F931F93FB016A01CB0165E0E7
:100B500070E00E94D030EF30F10538F48E2FE9308C
:100B6000F10508F088E0482F01C04E2FCF0196957F
:100B70008795969587954801590175E0E72E0AE01B
:100B8000262F682F81E08E0F0E9416221F910F9151
:100B9000EF90DF90CF90BF90AF909F908F9008958F
:100BA0002F923F924F925F926F927F928F929F927D
:100BB000AF92BF92CF92DF92EF92FF920F931F936B
:100BC000CF93DF93CDB7DEB729970FB6F894DEBF8A
:100BD0000FBECDBF6B012A0149013801CB0101963F
:100BE0008232910510F081E290E08887C60167E0CB
:100BF00070E00E94D0306987C60163E070E00E9417
:100C0000D0306E836B3010F08AE08E83C601880F7F
:100C1000991F63E070E00E94D0306B3008F06AE00A
:100C2000262E312C9E81291A3108EFEF2E1A3E0A0A
:100C3000E12CF12C86EFA82EBB24BA94EF82E88534
:100C4000EE1608F04AC0FBEAEF9E812D112486952E
:100C5000982F990F890F8E1106C08CE1C816D10408
:100C600020F4298503C020E001C023E0C701B101C1
:100C70000E94E4304E81480F7A2DBD82AC8290E410
:100C8000299F9001112484E0489FF0011124EF5620
:100C9000F74F51815F73522B5A834F704983830101
:100CA000940160E09AE0A91AB1088D810E94E021C8
:100CB000F201868D823018F0FF81F0FF04C08FEFC3
:100CC000E81AF80ABBCF8301940149815A8161E097
:100CD0007C818D810E94E021F2CF29960FB6F89495
:100CE000DEBF0FBECDBFDF91CF911F910F91FF905F
:100CF000EF90DF90CF90BF90AF909F908F907F90BC
:100D00006F905F904F903F902F900895CF93DF9317
:100D1000CDB7DEB727970FB6F894DEBF0FBECDBFB5
:100D2000FC0120812E3039F481810E94A2222650BC
:100D300081E0223008F080E027960FB6F894DEBFFD
:100D40000FBECDBFDF91CF9108950F931F93CF9327
:100D5000DF93CDB7DEB727970FB6F894DEBF0FBE8F
:100D6000CDBF062FFC011081812F0E94A2228F830C
:100D7000701302C017FD07C08F81801306C016FBD9
:100D8000882780F903C081E001C080E027960FB674
:100D9000F894DEBF0FBECDBFDF91CF911F910F91B1
:100DA00008950F931F93CF93DF93CDB7DEB72897A6
:100DB0000FB6F894DEBF0FBECDBF8C01FC01808161
:100DC0000E94A22262E0C80138870E94A5063885E9
:100DD000882321F0832F8695869501C080E0830FBC
:100DE00028960FB6F894DEBF0FBECDBFDF91CF912E
:100DF0001F910F910895FC0190819770673031F435
:100E0000923080F081E0943081F40CC0643021F4A1
:100E100081E0913051F406C06A3031F4965081E09F
:100E2000923018F080E0089581E00895FC01660F8B
:100E3000660F660F972F990F990F990F8081865033
:100E4000823020F084E0860F9C5F08958CEF860F3F
:100E500094500895DC0182E08093A40580E480939F
:100E6000900084E59DE090939900809398001196FE
:100E70009C9111979295969596959370E9F0EC91C7
:100E8000EF70E630C9F044E0E49FF0011124EF5622
:100E9000F74F818191509F7340E4949F90011124FA
:100EA0008F73282B11962C93119786EF9FEF149632
:100EB0009C938E931397089511961C9208959F9278
:100EC000AF92BF92CF92DF92EF92FF920F931F9358
:100ED000CF93DF93CDB7DEB727970FB6F894DEBF79
:100EE0000FBECDBF7C018B016A01922EDB016C919C
:100EF0006F700E94FB06B82E882309F481C0F701A9
:100F000080818770823091F063E0C7010E94A5065E
:100F1000B82E882359F00E943B3063E070E00E94B5
:100F2000E430BB24B394892B09F0B12CD7018C9108
:100F30000E94A222A52E60E0C7010E94A506882378
:100F400019F08A2D869501C080E0A80E8A2D90E0C8
:100F5000911003C061E070E002C062E070E00E94A6
:100F6000E430F8018181982F9F736917C8F0C80198
:100F70000E942A07D801EC91EF70B4E0EB9FF001DA
:100F80001124EF56F74F2381F60180819181820F62
:100F9000911D918380838FEFD70111968C9319C097
:100FA000961B292F2F73982F907C922BF8019183F9
:100FB000BB2079F08081282F2F70233011F09FE023
:100FC00001C097E0F0E19F9FC0011124822BD8015E
:100FD0008C93F70180818770863091F40E943B30BA
:100FE0006AE070E00E94E430892B51F4D801139636
:100FF0008D919C9114970A9714969C938E931397B6
:1010000027960FB6F894DEBF0FBECDBFDF91CF910C
:101010001F910F91FF90EF90DF90CF90BF90AF9016
:101020009F9008950F931F93CF93DF93DC01139646
:10103000ED91FC91149712968C91DB019FE0899FB2
:10104000A00DB11D11248C91880F880F880F8C5F23
:1010500011969C911197990F990F990F9C5FF7FD2D
:101060005CC050E018EF5A3018F4252F30E002C071
:1010700029E030E0ED01C20FD31F2D81322F3295D0
:10108000369536953370313039F070F0323039F0B2
:10109000333039F030E009C030E041E007C031E0E2
:1010A00004C030E04FEF02C03FEF40E02F73120367
:1010B000B00111246E0F7F1F77FF23C08F0123E043
:1010C000169507952A95E1F728EF2003B001219F97
:1010D000700D1124E60FF71F242F220F220F220F6D
:1010E000209F800D11244E9F800D1124232F220F4D
:1010F000220F220F209F900D11243E9F900D11244E
:101100000CC0220F220F220F429F800D1124329F0C
:10111000900D11245F5FFB01A6CFDF91CF911F914E
:101120000F9108952F923F924F925F926F927F920C
:101130008F929F92AF92BF92CF92DF92EF92FF92E7
:101140000F931F93CF93DF93CDB7DEB7C859D10963
:101150000FB6F894DEBF0FBECDBF46E056E0CC56CA
:10116000DF4F59834883C459D0402A01812C912CE8
:10117000CD56DF4F1882C359D040CE56DF4F18826C
:10118000C259D040F12C5FEFC557DF4F5883CB5881
:10119000D040140188E0281A31086201A12CB12C3A
:1011A00010E0D6018E913D018E3039F18091D70546
:1011B000813009F087C080918808811383C08091B5
:1011C00089088F117FC060918A08683008F07AC062
:1011D000809181089091820803E0969587950A9501
:1011E000E1F783709927892B09F46CC0CE01019631
:1011F0000E941C238981811165C0F30180818E309A
:1012000061F4D6018C910E94A22229833A834B83F8
:101210005C836D837E838F8325C0E0918A08B7E06D
:10122000BE9FF0011124EB5DFE4FDE01119687E0B9
:1012300001900D928A95E1F7EA81C557DF4FE88367
:10124000CB58D040612F7F2DCE0101960E9416070A
:10125000CD56DF4F8883C359D040CE56DF4F988399
:10126000C259D0408981863088F0863011F082E002
:1012700001C080E0D6014C91441F4427441F480F11
:10128000B101C50108970E944B182CC0612C712C2C
:1012900030E0332309F4C9C5F601808190E0313094
:1012A00019F040E450E002C040E850E08423952368
:1012B000892B09F4BAC53F5FF8E06F0E711C33301B
:1012C00041F710C0D3014C91B8E04B9FA00111240D
:1012D0004A525D4FEE24E39408E028E0B401C501D2
:1012E0000E94661F1F5FE8E0AE0EB11CF3E0CF0E58
:1012F000D11C103109F055CFF39428E0820E911CD7
:1013000040E3440E511C58E0F51243CFCF56DF4F57
:101310001882C159D040CC56DF4F48815981C459F9
:10132000D040C757DF4F59834883C958D040C05772
:10133000DF4F1882C059D040C757DF4FE881F9818D
:10134000C958D040319780818E3009F01CC2C757F0
:10135000DF4FA881B981C958D0401196EC91EF3F79
:1013600009F411C2B5E0BE9FF0011124EB57F84F0C
:10137000DE01959685E001900D928A95E1F78EA1A8
:101380008F7309F400C268ED75E0CE0185960E9466
:1013900012084C01C757DF4FE881F981C958D04086
:1013A0008081982F9873E92EF12C270113E0559432
:1013B00047941A95E1F7FCE0F49DA02C11240E94BB
:1013C000A22229833A834B835C836D837E838F8340
:1013D000C057DF4F6881C059D040CF56DF4F78816A
:1013E000C159D040CE0101960E9416073C01282C1D
:1013F000312C082F10E0A101401B510BC457DF4FC7
:1014000059834883CC58D0402A2D30E0429FC001F8
:10141000439F900D529F900D112464E670E00E944E
:10142000E430B62CB60EC92CD12CE72CF12CF601E9
:10143000EE19FF09C257DF4FF983E883CE58D04039
:10144000E29FC001E39F900DF29F900D112464E68E
:1014500070E00E94E430372D360FC757DF4FA88168
:10146000B981C958D040EC91E7708E2F90E0FC0113
:101470003197E730F105D0F4EA5AFF4F0C94F83079
:10148000C20101964C01880C991C880E991E712C82
:101490007201B2E0EB0EF11C032F10E002501109B3
:1014A000CB2CD12CE2E0CE1AD10850C1861418F40E
:1014B0000219130906C0C457DF4F08811981CC589F
:1014C000D040971418F4EC18FD0806C0C257DF4F3F
:1014D000E880F980CE58D040E016F1065CF4303454
:1014E00008F051C1632F70E042E08B2D90E00E9424
:1014F000E41749C1632F70E020E042E08B2D90E0BB
:101500000FC0032F10E0EB2CF12C20E042E0B801DB
:10151000C70101970E94982520E042E0B801C70169
:101520000E94982530C1E32EF12C0B2D10E020E015
:10153000A701B80184EC95E00E94D3205701FFEF8A
:10154000AF1ABF0A68012FEFC21AD20A20E0A50124
:10155000B60184EC95E00E94D3200150110920E0EF
:10156000A501B80184EC95E00E94D32041E0E41A83
:10157000F10820E0A701B60184EC95E00E94D32099
:1015800020E0A701B80184EC95E00E94D320FBC0C5
:10159000EB2DF0E0C32ED12CEC18FD0859E15E9D37
:1015A000C0015F9D900D112464E670E00E94E4305C
:1015B000630F262F30E00E1B1F0BA9E1A09FC00177
:1015C000A19F900D112464E670E00E94E430B60EF5
:1015D0004B2D50E0B601CF0122C0632F70E041E0F7
:1015E0008B2D90E00E948318CEC0B1E3BA1508F4A9
:1015F000CAC080918108909182089C012370332792
:101600002C0D3D1D2150310963E070E00E94D03067
:10161000A101480F591F41505109B701C8010E944B
:101620006519B1C0E42CE694E394632E712C0B2D64
:1016300010E0CE2CD12CEE0C41E04E0DB3016C1914
:101640007D0920E0C8010E949825EE24E394F12C46
:10165000EC18FD08222433242C183D08220C331CDE
:1016600044244394512C812C912CC257DF4F198371
:101670000883CE58D040CA56DF4F79826882C65957
:10168000D040F7FC08C0E1E0CE1AD108F2E02F0EFE
:10169000311CE20CF31C2FEF821A920A42E0440E36
:1016A000511CE40CF51C8C2D880F31E0380F20E024
:1016B000432FC3018C199D09C457DF4F9983888339
:1016C000CC58D040BC01C257DF4F88819981CE5899
:1016D000D040880D991DC856DF4F3883C859D04077
:1016E0000E949825CA56DF4FA880B980C659D040BD
:1016F000A818B90820E0442DB501C8018C0D9D1D26
:101700000E94982520E0C856DF4F3881C859D04044
:10171000432FC457DF4F68817981CC58D040C257DE
:10172000DF4F88819981CE58D040881999090E944D
:10173000982520E0442DB501C8018C199D090E940F
:1017400098258C149D040CF49CCF1DC0872D90E02F
:1017500088159905C4F40E943B30B7010E94E4301B
:101760005801A80EB91E0E943B30B7010E94E43018
:10177000B601680F791F20E0A50184EC95E00E9476
:10178000D3207394E3CFC057DF4F9881C059D04026
:101790009F5FC057DF4F9883C059D040C757DF4F76
:1017A000A881B981C958D0401396C757DF4FB98374
:1017B000A883C958D040903109F0BECDCF56DF4F35
:1017C000B881C159D040BF5FCF56DF4FB883C159F0
:1017D000D040CC56DF4FE881F981C459D040F09613
:1017E000CC56DF4FF983E883C459D040B83009F0B4
:1017F00092CD10E075E0D72EE4E26E2EE2E07E2E70
:10180000F5E2AF2EF2E0BF2EA2E08A2E912C812FBE
:1018100090E020917F08309180088217930708F0AC
:101820006FC0D89E9001D99E300D1124C9018B57ED
:10183000984F2C01DC0113968D919C91149797FD84
:101840005DC011968C918F7309F458C068ED75E0F6
:10185000C2010E941208F82E692FD201EC91EF709C
:10186000B4E0EB9FF0011124EF56F74F2081F20115
:1018700043815481F3010491F501E490222309F49A
:10188000F0C230E0220F331FE02FF0E08E2D86955E
:1018900086958695A82FB0E081E090E07E2D777048
:1018A00011F480E090E08A0F9B1FE89FD001E99F30
:1018B000B00DF89FB00D11242A9FF0012B9FF00D61
:1018C0003A9FF00D1124EA5DFD4F70E09B0124501A
:1018D0003109CA019595879595958795B4010E9420
:1018E000E430B901680F711D8F2D90E023E0C22E06
:1018F00020E030E0AF0104970E94671D1F5F87CF93
:10190000E0908908EE0CEE0CEE0C00918808000FB8
:10191000000F000FF12C10E028E048E0B701C801EB
:101920000E941B185801B8E0AB0EB11CC12CD12C81
:1019300063E0262E312C2801E7E04E0E511C4701B2
:10194000F7E08F0E911C3701601A710A80918108AF
:101950009091820853E0969587955A95E1F78C0D02
:101960009D1DB1010E94D030892B11F521E0A70106
:10197000B601600F711F84EC95E00E94D32021E036
:10198000A6014E0D5F1DB20184EC95E00E94D320AC
:1019900021E0A401B50184EC95E00E94D32021E070
:1019A000A3014A0D5B1DB80184EC95E00E94D32091
:1019B0002FEFC21AD20A41E0A41AB10858E0C516A6
:1019C000D10421F68091D705813021F00E94531F68
:1019D00082FD62C08091D705813009F445C28091B3
:1019E0008908811141C208E31092D30581E08093F8
:1019F000D40510E081E090E09093D0058093CF056E
:101A00001093D2050093D10564E280EC95E00E942A
:101A1000F12080910306813009F028C261E280EC58
:101A200095E00E94F12061E280EC95E00E94F120B7
:101A300061E280EC95E00E94F12089E290E09093D1
:101A4000D0058093CF051093D2050093D1056CE4A7
:101A500080EC95E00E94F1206091850870918608E5
:101A600080E090E04AE00E94572589E590E090935D
:101A7000D0058093CF051093D2050093D10562E580
:101A800080EC95E00E94F1206091870870E080E092
:101A900090E04AE00E9457258091D705833009F0F5
:101AA0005CC00E94531F83FF58C010E045E0D42E55
:101AB000812F90E020917F08309180088217930752
:101AC00008F04BC0D89EF001D99EF00D1124EB57C1
:101AD000F84FDE0111968D2D01900D928A95E1F758
:101AE0008C819D8197FD37C08A818F73A1F168ED4C
:101AF00075E0CE0101960E941208E981EF7024E0A2
:101B0000E29FF0011124EF56F74F9180CA80A92E71
:101B1000B12CE82EF12CB5016650710901E023E0EB
:101B200046E0C70103970E94C4259501255031095D
:101B30002034310580F48C2D8F73A5E08A9FC0017D
:101B40001124692D70E00E94D030462FB901C701E1
:101B500002970E94E4171F5FABCF00918808809125
:101B600089089091D705913009F0AAC010E0B0E142
:101B70008B9F000D111D1124C801880F991F080F9C
:101B8000191FF801E952FA4F86A58E3009F098C066
:101B900008521A4F7801EEE2EE0EF11CC7010E94C6
:101BA000D106C557DF4F8883CB58D04064E0C701CA
:101BB0000E94A506F82E8091810883FD62C0809165
:101BC0008A08883091F468E0CE01875B9F4F0E94BD
:101BD0001C232A968FAD2A97811107C0D8019E96A3
:101BE0008C910E94A222723091F080918A088930F3
:101BF00009F569E0CE0101960E941C2389818111BB
:101C000019C0F80186A50E94A222823099F4C55716
:101C1000DF4F8881CB58D04086958695C557DF4FDA
:101C2000F881CB58D040F80FC557DF4FF883CB5819
:101C3000D04027C080918A08883079F468E0CE01CE
:101C400085960E941C238DA1811107C0D8019E9604
:101C50008C910E94A222743091F080918A08893080
:101C600081F469E0CE0101960E941C2389818111D3
:101C700008C0F80186A50E94A222843011F4FF2436
:101C8000F394D8019E968C910E94A22229833A83D4
:101C90004B835C836D837E838F8360918808709112
:101CA0008908CE0101960E941607CD56DF4F888322
:101CB000C359D040CE56DF4F9883C259D04001C09F
:101CC000F12CC557DF4FB881CB58D040BF3FF1F062
:101CD000CE56DF4FE881C259D0400E2F10E0CD56CE
:101CE000DF4FF881C359D040CF2ED12C4B2FB801F4
:101CF000C6010E948318FF2049F0B8016C50710999
:101D000028E148E1C6010C970E941B188091D70575
:101D1000813009F0B5C001E029E040E867E370E0F8
:101D200080E090E00E94C42540E867E370E080E036
:101D300090E00E94E417C12CD12C10E082E0F82E34
:101D4000AA24A394B12C2FE2822E912C1D3030F4C2
:101D5000612FCE0101960E941C2302C0F9821D82D0
:101D60008981823009F48CC080918A08811335C042
:101D70004A815B81E12C08E028E068E370E0C6015D
:101D80000E94661FB092D005A092CF059092D20516
:101D90008092D105CE0105960E9445258C8188232D
:101DA00079F160E280EC95E00E94F12068E280EC3D
:101DB00095E00E94F12064E280EC95E00E94F12021
:101DC0006C8170E080E090E04AE00E94572569E273
:101DD00080EC95E00E94F12013C000E028E048E08C
:101DE00068E370E0C6010E94C4254A815B81EE244D
:101DF000E39408E028E068E370E0C6010E94661FF3
:101E00008981813051F4E12C08E028E04CE152E076
:101E100068E370E0C6010E94661F1F5F28E0C20EE3
:101E2000D11C103109F092CF2BC08981A30198E118
:101E3000899F400D511D11244C58564FEE24E394B8
:101E400008E028E0B401C501C856DF4F3883C859FF
:101E5000D0400E94661FC856DF4F3881C859D04015
:101E60002ACAE6E2F2E031CD01E0BECD60918308FE
:101E70007091840880E090E04AE00E945725DDCD13
:101E8000C856DF4F0FB6F894DEBF0FBECDBFDF914F
:101E9000CF911F910F91FF90EF90DF90CF90BF9067
:101EA000AF909F908F907F906F905F904F903F90FA
:101EB0002F900895FC0182818A3070F4DF01A80F11
:101EC000B11D15966C936F7323813481260F311DDC
:101ED000348323838F5F82830895FC0110821182F3
:101EE000DC0115960F9621E02D93A817B907E1F7AD
:101EF000108211821282148213820895E92F572FC3
:101F0000A82FB0E0262F30E0681720F4CD01821B07
:101F1000930B03C0C9018A1B9B0B6E2F70E0252F0A
:101F200030E05E1728F4FB01E21BF30B9F0102C0B7
:101F3000261B370B50E048175907B8F142175307D3
:101F4000A0F1229FB001239F700D700D1124889F76
:101F50009001899F300D300D1124260F371F80E02E
:101F600090E42817390728F49695879596958795D4
:101F7000F8CF60E070E0009791F0FC01E60FF71FEA
:101F80002E173F0728F02E1B3F0BBF01680F791F4C
:101F9000969587959695879576956795ECCF81E090
:101FA0004617570718F080E0089581E00895EF92F2
:101FB000FF920F931F93CF93DF931F92CDB7DEB79E
:101FC0007C01FC0100811181C80169830E944B30B2
:101FD0006981681719F0C8010E945330C7010F903A
:101FE000DF91CF911F910F91FF90EF9008952F9265
:101FF0003F924F925F926F927F928F929F92AF9299
:10200000BF92CF92DF92EF92FF920F931F93CF93E5
:10201000DF93CDB7DEB7E3970FB6F894DEBF0FBE00
:10202000CDBF9091D705923089F038F4992309F407
:1020300073C1913009F488C0DEC5943009F479C5C4
:1020400008F453C0953009F4C3C5D5C5883009F0EC
:102050004CC081E08093D705D09088082EE02D15E4
:1020600008F4C9C510918908173008F0C4C501E00B
:102070000D0DE02EF12CC70130E1139F800D911D55
:1020800011249C01220F331F820F931F8B5F994FE6
:102090000E948606882319F000938808ACC51F5F4C
:1020A00070E1179F5001112495012D0D311DC901BB
:1020B000880F991F820F931F8B5F994F0E9486068E
:1020C000811110C0EA0CFB1CC701880F991F8E0DEF
:1020D0009F1D8B5F994F0E948606882309F48BC54C
:1020E000009388081093890886C5803231F118F46E
:1020F000803131F080C58034A9F0803861F07BC533
:1021000080918908282F30E02630310514F48F5F44
:1021100006C087E004C080918908811181508093B6
:10212000890869C580918808282F30E02E30310554
:1021300014F48F5F06C08FE004C08091880881117D
:1021400081508093880857C5883099F028F48430EE
:1021500009F051C582E0D7C0803209F4D7C080347D
:1021600009F049C580918A0890E001966DE070E021
:10217000E1C060918A086D3008F03DC5CE0101963E
:102180000E941C238981811136C560918A086830BC
:1021900008F045C0CE0101960E941C238981813040
:1021A000F1F180918A0897E0899FF0011124EB5D9D
:1021B000FE4F448150E02091830830918408241719
:1021C000350720F490910306913049F5241B350B17
:1021D000309384082093830890918908E0918808BF
:1021E000F0E0A0E19A9FE00DF11D11249F01220F64
:1021F000331FE20FF31FE952FA4FDF019E969EE074
:1022000096A7877011968C9311978FEF12968C93E7
:1022100082E08093D70510928A080E94CB22F0902A
:102220008A08BAE0FB1609F46CC0BF1520F0E8E09C
:10223000FE1650F4E0C4FBE0FF1609F44CC02CE09D
:10224000F21609F45EC0D7C480918908009188080D
:1022500010E030E1839F000D111D11246801CC0CAA
:10226000DD1CF601E00FF11FEA5FF94F80810E944B
:10227000A222862F90E0880F991F63E070E00E94F1
:10228000E43080918308909184088617970728F49A
:1022900080910306813009F0AEC4F601E00FF11F12
:1022A000E852FA4F86A598E0F91611F090E401C0C3
:1022B00090E80C0D1D1DF801E852FA4F892B86A7F6
:1022C0008091830890918408861B970B90938408D3
:1022D0008093830890C48091F7059091F805DC0104
:1022E000ED91FC916091870870E00190F081E02D04
:1022F0000FE718E025E837E048ED55E0099583E061
:1023000002C084E062C48093D70520C480918A080B
:10231000811117C08CE018C0803279F0803421F030
:10232000883009F068C413C080918A0890E0019653
:1023300066E070E00E94E43007C080918A0888233C
:1023400011F0815001C085E080938A0854C4109137
:102350008A08153008F0E3C31092800810927F08B5
:1023600010928408109283081092870810928608B1
:1023700010928508CE0185960E946D0FCE010196C0
:102380000E946D0F1092F605123009F4E3C020F49C
:10239000113009F44AC006C0133009F45CC114308E
:1023A00009F4EEC181E08DA38EA365E8CE01859688
:1023B0000E945A0F62E4CE0185960E945A0F65E092
:1023C000CE0185960E945A0F68E4CE0185960E9440
:1023D0005A0F62E8CE0185960E945A0F65ECCE0135
:1023E00085960E945A0F63E8CE0185960E945A0F87
:1023F00067E4CE0185960E945A0F65E0CE0185966E
:102400000E945A0FADA0BEA0CFA0D8A4E9A4FAA400
:102410000BA51CA52DA53EA54FA558A969A97AA96C
:102420008BA90E94E62584E18DC011E01DA31EA3A7
:1024300062E8CE0185960E945A0F67E4CE01859628
:102440000E945A0F61E8CE0185960E945A0F62E4FD
:10245000CE0185960E945A0F62E8CE0185960E94B1
:102460005A0F64E4CE0185960E945A0F63E0CE01B4
:1024700085960E945A0F62ECCE0185960E945A0FF3
:1024800062E0CE0185960E945A0F64ECCE018596DB
:102490000E945A0F198386E08A8363E0CE01019679
:1024A0000E945A0F63E4CE0101960E945A0F62E81F
:1024B000CE0101960E945A0F61E4CE0101960E945E
:1024C0005A0F61E8CE0101960E945A0F69E4CE01CD
:1024D00001960E945A0F63E0CE0101960E945A0FA6
:1024E00062ECCE0101960E945A0F62E0CE01019685
:1024F0000E945A0F64ECCE0101960E945A0FADA0C3
:10250000BEA0CFA0D8A4E9A4FAA40BA51CA52DA514
:102510003EA54FA558A969A97AA98BA90E94E625CD
:10252000A980BA80CB80DC80ED80FE800F81188589
:1025300029853A854B855C856D857E858F850E94D2
:10254000E62589E18093F9058AE08093FA058BEF0F
:1025500095E0A5C111E01DA31EA365E8CE018596F7
:102560000E945A0F62E4CE0185960E945A0F62E0E3
:10257000CE0185960E945A0F62E4CE0185960E9494
:102580005A0F62E8CE0185960E945A0F63E4CE018D
:1025900085960E945A0F63E0CE0185960E945A0FDD
:1025A00062ECCE0185960E945A0F62E0CE018596BC
:1025B0000E945A0F63ECCE0185960E945A0F8EE05E
:1025C00089831A8364ECCE0101960E945A0F65E854
:1025D000CE0101960E945A0F62E4CE0101960E943C
:1025E0005A0F63E0CE0101960E945A0F62E4CE01B9
:1025F00001960E945A0F63E8CE0101960E945A0F7D
:10260000ADA0BEA0CFA0D8A4E9A4FAA40BA51CA598
:102610002DA53EA54FA558A969A97AA98BA90E9405
:10262000E625A980BA80CB80DC80ED80FE800F811A
:10263000188529853A854B855C856D857E858F85D6
:102640000E94E62584E18093F9058AE08093FA05EB
:102650008DEF95E024C102E00DA317E01EA362E018
:10266000CE0185960E945A0F6CE4CE0185960E9499
:102670005A0F62E8CE0185960E945A0F67ECCE0190
:1026800085960E945A0F66E0CE0185960E945A0FE9
:1026900062ECCE0185960E945A0F62E8CE018596C3
:1026A0000E945A0F64ECCE0185960E945A0F61E099
:1026B000CE0185960E945A0F63E4CE0185960E9452
:1026C0005A0F09831A8362E0CE0101960E945A0FC5
:1026D0006CE4CE0101960E945A0F62E8CE01019689
:1026E0000E945A0F67ECCE0101960E945A0F66E0D5
:1026F000CE0101960E945A0F62E4CE0101960E941B
:102700005A0F62E8CE0101960E945A0F64E4CE018E
:1027100001960E945A0F61E0CE0101960E945A0F65
:1027200063ECCE0101960E945A0FADA0BEA0CFA0CF
:10273000D8A4E9A4FAA40BA51CA52DA53EA54FA5D8
:1027400058A969A97AA98BA90E94E625A980BA800F
:10275000CB80DC80ED80FE800F81188529853A854D
:102760004B855C856D857E858F850E94E6258AE098
:102770008093F90588E08093FA058FEF95E08FC08C
:102780001DA31EA362E0CE0185960E945A0F63EC42
:10279000CE0185960E945A0F64E8CE0185960E946C
:1027A0005A0F65E4CE0185960E945A0F65E0CE016E
:1027B00085960E945A0F62E4CE0185960E945A0FB8
:1027C00065E8CE0185960E945A0F63E4CE01859696
:1027D0000E945A0F65E0CE0185960E945A0F63E46D
:1027E000CE0185960E945A0F8DE0898386E08A8308
:1027F00063E0CE0101960E945A0F65ECCE0101966E
:102800000E945A0F63E8CE0101960E945A0F62ECB3
:10281000CE0101960E945A0F63E0CE0101960E94FC
:102820005A0F61ECCE0101960E945A0F62E0CE0170
:1028300001960E945A0F63ECCE0101960E945A0F36
:1028400063E8CE0101960E945A0FADA0BEA0CFA0B2
:10285000D8A4E9A4FAA40BA51CA52DA53EA54FA5B7
:1028600058A969A97AA98BA90E94E625A980BA80EE
:10287000CB80DC80ED80FE800F81188529853A852C
:102880004B855C856D857E858F850E94E6258EE172
:102890008093F90586E18093FA0581E096E09093B4
:1028A000F8058093F70580E090E02FEFFC01E952F6
:1028B000FA4F16A617A620AB03968038B1E09B0707
:1028C000A9F720E0EFE05E2E6624639422242A9488
:1028D000F2E07F2E8091F605281708F0FFC0223025
:1028E00018F4822F90E002C081E090E0589EA00191
:1028F000599E500D1124FA01E952FA4F7F018F01C0
:102900000F5F1F4F8181D80111966C9130E0A1E0DB
:102910005A01F8019281391708F0AFC03A3018F423
:10292000432F50E002C049E050E04A0D5B1DFA0120
:10293000E352FA4FE0819E2F92959695969593706B
:10294000913041F060F0923041F040E0933041F43A
:102950005FEF07C040E051E004C041E001C04FEF2D
:1029600050E0A111892E912CEF734E2E941408F093
:1029700081C0E82FF0E0B0E16B9FE00DF11D112464
:102980006F01CC0CDD1CD601AE0FBF1FA952BA4F90
:102990009E96BC91992371F172E0871601F1AB2FDD
:1029A000AB7FA33031F0B53021F0A5EFAB0FA330F2
:1029B00010F478E001C070E09130A9F0A3E08A162D
:1029C00091F0ACEFAB0FA33070F0A7EFAB0FA230DC
:1029D00050F0A4EFAB0FA23030F0A0E005C0913072
:1029E00009F007C178E0A4E0A72B923099F0882085
:1029F00089F004C073E08712FCC0ACE0B33051F042
:102A0000B63041F078EF7B0F743020F0BD3011F01C
:102A100070E001C072E0372E3A2A933079F071E00D
:102A2000871661F0B43051F0A9EFAB0FA23030F04F
:102A3000BA50A1E0B43018F0A0E001C0A1E0A32991
:102A4000A350AD3028F4B0E0AF5EBE4F8C9001C013
:102A5000812CEC0DFD1DE952FA4FDF019E9686A6F2
:102A600011961C92119712962C929394850F640FD5
:102A7000892E7CCF3F5FA0E04CCF9181D70111968A
:102A8000EC91F0E0B0E19B9FE00DF11D1124AF014E
:102A9000440F551FE40FF51FE952FA4FDF019E96D0
:102AA00066A611961C92119712962C9290E0E0E186
:102AB0006E9F800D911D1124FC01EE0FFF1F8E0FE4
:102AC0009F1FFC01E952FA4FDF019E9676A61196F0
:102AD0001C92119712962C922F5FFCCE80918A083F
:102AE00080930406109287088091FA0590E09093F5
:102AF0008408809383088091F90590E0909386087C
:102B00008093850888E08093880884E08093890812
:102B100010928A0880E090E00E94403055C0153045
:102B200009F069C090918B0881E0892780938B0818
:102B300062C0843011F481E048C0883009F05BC085
:102B400080918A088C3029F41092D70510928A0857
:102B500052C08A3009F04FC08091890800918808DE
:102B600010E0F0E18F9F000D111D1124C801880FA6
:102B7000991F080F191FF801EA5FF94F80810E9421
:102B8000A22266958091830890918408860F911DFA
:102B90009093840880938308F801E952FA4FDF018B
:102BA0009E9616A611961C9211978FEF12968C93F3
:102BB00085E08093A40580E4809390008CE195E10A
:102BC000909399008093980082E08093D70513C07A
:102BD000883011F0843079F480918708E091040600
:102BE000F0E0E457F74F9081981708F0ADCF80835D
:102BF000ABCF78E0E6CEE3960FB6F894DEBF0FBE1B
:102C0000CDBFDF91CF911F910F91FF90EF90DF909B
:102C1000CF90BF90AF909F908F907F906F905F907C
:102C20004F903F902F90089580E0E4EAF1E0811109
:102C30008FEF002481938193819381930394D1F743
:102C4000E0ECF5E0128A118A108A17860895E4EA0A
:102C5000F1E0A0E0B8E000800EBC8111012C1197DA
:102C6000A0FDFDCF0192B9F70DB40895FC0180914C
:102C7000AD05811103C08FEF9FEF08959FB7F894C2
:102C800082E08093E9002091F20030E012161306F2
:102C900014F421E030E02115310559F0289884E63C
:102CA0008093AC058091F10080838091F2008823AD
:102CB00019F09FBFC90108958BE68093E800F9CF12
:102CC0002FB7F89483E08093E9009091E800892F72
:102CD000807295FF04C09091F20080E4891B2FBFA1
:102CE00008958091B30581110DC082E08093AF05F6
:102CF00084E08093B0051092B2051092B10581E096
:102D00008093B3058FEA95E00895CF93DF931F92E8
:102D1000CDB7DEB76983DC01ED91FC910280F381D0
:102D2000E02D41E050E0BE016F5F7F4F09950F90AD
:102D3000DF91CF91089583E08093E9008091F200C4
:102D4000882319F08AE38093E80008950E946016B2
:102D500090E00895CF93DF931F92CDB7DEB7FC01CB
:102D60008485958597FD05C02FEF3FEF3587248734
:102D70000BC0CE0101960E943616019719F4898185
:102D800090E002C08FEF9FEF0F90DF91CF910895F9
:102D90000F931F93CF93DF931F92CDB7DEB78C01B4
:102DA000FC018485958597FF0EC0CE0101960E9497
:102DB0003616019719F4298130E002C02FEF3FEF5A
:102DC000F80135872487F801848595850F90DF9178
:102DD000CF911F910F910895FC018485958597FDF2
:102DE0000BC09FB7F89482E08093E9008091F200D5
:102DF0009FBF90E0019608959FB7F89482E080937A
:102E0000E9008091F2009FBF90E008958F929F9219
:102E1000AF92BF92CF92DF92EF92FF920F931F93E8
:102E2000CF93DF935C016B017A0180910B018823C2
:102E300009F45BC08091AD05882309F456C08091E8
:102E4000AB0580FF05C08091E00082608093E000C8
:102E5000E70110E00AEF83E0882E9AE3992E20978D
:102E6000D9F10E94601681110AC0015009F43DC0D9
:102E700061E070E080E090E00E94E31CF0CF282F3A
:102E800030E0C217D3070CF48C2F4FB7F894809220
:102E9000E9009091E80095FF1DC0282F30E0C21B8B
:102EA000D30BF601982F915020F081918093F1007F
:102EB000FACFC20ED31E112319F09092E80009C078
:102EC0008091E80085FD06C09092E80011E020970F
:102ED00009F010E04FBFC3CF1111C3CF5D9884E656
:102EE0008093AE051E141F0444F081E090E0F501CC
:102EF0009383828380E090E001C0C701DF91CF918E
:102F00001F910F91FF90EF90DF90CF90BF90AF9007
:102F10009F908F900895DF92EF92FF920F931F93EF
:102F2000CF93DF93D82E8A017B01E40EF51EEB01CF
:102F3000CE15DF0571F0D7FE03C0FE01849101C0FC
:102F400088810E942B2621968111F2CF8FEF9FEF6F
:102F500001C0C801DF91CF911F910F91FF90EF90B9
:102F6000DF9008950F931F93CF93DF931F92CDB7F8
:102F7000DEB782E0898342E450E066E473E080E8F3
:102F80000E948B170E947116DC0112960D911C9104
:102F900013970115110569F0D801ED91FC9102809C
:102FA000F381E02DBE016F5F7F4FC801099597FF48
:102FB00007C089810F90DF91CF911F910F910895E4
:102FC000F80100851185E5CF9C01240F311D1216F3
:102FD000130684F5803891056CF5FC0197FF02C05B
:102FE000E0E0F0E02138310514F020E830E02E1B5D
:102FF000AB014770552781E090E001C0880F4A95EA
:10300000EAF7809577FF02C0695F7F4F93E075957F
:1030100067959A95E1F77695762F66277795679568
:10302000E60FF71FEC55FE4F215020F090819823BA
:103030009193FACF0895EF92FF920F931F93CF933E
:10304000DF93EC018B01E42EF22E6034710510F455
:103050000E94E417B8016F0D711D61507109603451
:10306000710520F44E2DCE010E94E41720E04F2D73
:10307000B801CE010E949825CE018E0D911D20E051
:103080004F2DB8010197DF91CF911F910F91FF90C4
:10309000EF900C949825CF92EF920F93E2EBF3E030
:1030A0000491E3EBF3E0E490442309F1A02FB0E0B6
:1030B0002E2D269526952695E22FF0E021E030E092
:1030C0005E2D577011F420E030E02E0F3F1FA29FBD
:1030D000F001A39FF00DB29FF00D11244E9F9001BF
:1030E0004F9F300D1124A9014C545C4F02C044EB9A
:1030F00053E022E0C22E20E030E00E94671D0F91D5
:10310000EF90CF9008952F923F924F925F926F92DF
:103110007F928F929F92AF92BF92CF92DF92EF9267
:10312000FF920F931F93CF93DF9300D000D0CDB7C2
:10313000DEB78C017B01242F30E03C832B8381E0C0
:1031400090E05C01A21AB30AC90191958195910999
:103150001C01220C331CA901460F571F20E0B801A7
:1031600084EC95E00E94D320A7018B819C81481BB1
:10317000590B20E0B80184EC95E00E94D3206B81CC
:103180007C81600F711F20E0A70184EC95E00E9414
:10319000D320B801EB81FC816E1B7F0B20E0A701DF
:1031A00084EC95E00E94D320C12CD12C21E030E0AA
:1031B0003A8329832B813C81C216D3060CF06EC062
:1031C000B7FC0AC08B819C8101979C838B8392E022
:1031D000290E311CA20CB31CEFEFCE1ADE0A298196
:1031E0003A812E5F3F4F3A832983A20EB31E3601E8
:1031F000600E711E20E08B809C808E0C9F1CA401B1
:10320000B30184EC95E00E94D32028014C185D089E
:1032100020E0A401B20184EC95E00E94D32020E0DC
:1032200047018B819C81881A990AA401B30184EC1F
:1032300095E00E94D32020E0A401B20184EC95E047
:103240000E94D32046018E0C9F1C20E0A4016B80BD
:103250007C80600E711EB30184EC95E00E94D32047
:1032600020E0A4012801EB81FC814E1A5F0AB20123
:1032700084EC95E00E94D32047018C189D0820E043
:10328000A401B30184EC95E00E94D32020E0A401C6
:10329000B20184EC95E00E94D3208CCF0F900F9068
:1032A0000F900F90DF91CF911F910F91FF90EF90B2
:1032B000DF90CF90BF90AF909F908F907F906F9056
:1032C0005F904F903F902F9008955F926F927F9202
:1032D0008F929F92AF92BF92CF92DF92EF92FF9226
:1032E0000F931F93CF93DF93EC018B017A01A90118
:1032F000461B570B57FF03C0519541955109C70114
:103300008C1B9D0B97FF03C09195819591095524C6
:1033100053948417950714F0512C0AC09E2D8F2DBD
:103320007901292F382F9C2F8D2FE801092F182F75
:10333000EC16FD0654F4902F812F8901292F382F88
:103340009C2F8D2FE701E92EF82E37016C1A7D0A8C
:103350005901A01AB10AB7FE03C0B194A194B108F3
:10336000630177FE03C08FEFC81AD80AD594C794BB
:103370000217130714F08FEF01C081E0882E880F29
:103380009908EC16FD06B4F020E0552019F0AE01C6
:10339000B80102C0A801BE0184EC95E00E94D320D0
:1033A000CA18DB08D7FE04C0080D191DC60CD71CAF
:1033B0002196E7CFDF91CF911F910F91FF90EF9072
:1033C000DF90CF90BF90AF909F908F907F906F9045
:1033D0005F9008951F920F920FB60F9211248F9352
:1033E0009F938091E1009091E100937F9093E100A1
:1033F00083FF0FC01092E90091E09093EB001092D0
:10340000EC0092E39093ED001092AD0598E090935C
:10341000F00082FF20C093E09093E9009091F200C9
:10342000992319F09AE39093E8009091AE059923BF
:1034300039F09091AE0591509093AE05992389F1A2
:103440009091AC05992339F09091AC0591509093EF
:10345000AC05992341F184FF10C08091E2008E7E7B
:1034600081608093E2008091E1008F7E8093E10093
:103470008091AB058E7E806111C080FF16C0809167
:10348000E2008E7E80618093E2008091E1008E7E7A
:103490008093E1008091AB058E7E81608093AB05C7
:1034A00004C05D9ACDCF289AD6CF9F918F910F906F
:1034B0000FBE0F901F9018951F920F920FB60F928C
:1034C0001124CF92DF92EF92FF920F931F932F93CD
:1034D0003F934F935F936F937F938F939F93AF939C
:1034E000BF93EF93FF93CF93DF93CDB7DEB76C9786
:1034F000DEBFCDBF1092E9008091E80083FFEDC1EF
:1035000068E0CE0145960E94592682EF8093E8003C
:103510008D8987FF05C09091E80090FFFCCF03C024
:103520009EEF9093E800982F907609F0C6C09E8990
:103530002F89188D91110CC0803829F48091AA052B
:103540008093F10002C01092F1001092F10048C186
:10355000422F50E0512B913051F4811141C1413043
:10356000510509F03DC18091AA058D7F0BC09330B4
:1035700061F4811135C14130510509F031C18091AB
:10358000AA0582608093AA052BC1953041F48091F1
:10359000E80080FFFCCF20682093E30021C1963033
:1035A00009F05FC0EB8CFC8C1092E9001092A8052A
:1035B0001092A705123091F51092A6051092A5055C
:1035C0000E94B21799E0BE016F5F7F4FDB01E92FC8
:1035D0001D92EA95E9F799831A8391E09E8390EA18
:1035E00098879AEF99872091A7053091A805275FC2
:1035F0003F4F3C832B838D831092E9001092A805E6
:103600001092A705F092A605E092A50549E050E0CA
:1036100080E00E948B170E94B217E2C0F092A605CC
:10362000E092A5050E947116DC011296ED90FC90C7
:103630001397E114F10409F4C0C0D701ED91FC9196
:103640000480F581E02DBE016B5E7F4FC7010995B7
:10365000009719F00CF0C4C0C7C0F701E084F184F2
:10366000E8CF973009F4C0C0983021F481E080930E
:10367000F100B6C0993009F0B3C0837009F0B4C04E
:10368000EFE1F1E081E021E036E39081992361F000
:103690008093E9002093EB0091919093EC0030939C
:1036A000ED008F5F873089F78EE78093EA001092F4
:1036B000EA008F898093AD0593C08B8D9C8D10920D
:1036C000E9001092A8051092A7059093A605809393
:1036D000A505898D811156C08E899D89913A59F42D
:1036E000813209F081C047E050E064E071E080E0A1
:1036F0000E948B1775C0913209F076C0833289F42D
:10370000888D90E0982F88272F89822BA0E0B0E049
:103710008093000190930101A0930201B0930301F3
:103720005FC0803269F48091E80082FFFCCF67E0DF
:1037300084E091E00E9459268BEF8093E80006C058
:10374000823209F04DC08F8980930B018091A905C9
:10375000882319F0EEEFFAE002C0E0E0F8E0809193
:10376000040190910501A0910601B0910701803BF1
:103770009440A105B10509F07BC080910B0180FF49
:1037800093C076C00E947116DC0112960D911C91B7
:1037900013970115110541F1D801ED91FC910190AC
:1037A000F081E02DBE016B5E7F4FC801099581114C
:1037B00017C0F80100851185ECCF113009F44EC017
:1037C000133091F48F89882309F445C0823081F445
:1037D00040E867E08AEA93E00E943F2E882321F0C8
:1037E0008EEF8093E80079C081E28093EB0075C092
:1037F000813029F440E86BE08EE993E0EDCF83302F
:1038000099F70E947116DC011296ED90FC901397C7
:103810008E010F5F1F4F6801E114F10479F0D701A9
:10382000ED91FC910680F781E02DB801C701099563
:10383000080F111DF701E084F184EECFD8011C922E
:10384000F60101900020E9F73197BF016C197D095D
:1038500040E0C601C1CF68E873E002C06CE873E0E5
:103860006115710509F2FB01449150E080E840CFF9
:103870000FB6F894A89580916000886180936000ED
:10388000109260000FBEA895EE3F2AE0F20739F0D3
:103890008091FE0A9091FF0A91838083A1CF1092BC
:1038A000FF0A1092FE0A9CCFEE3F8AE0F80731F043
:1038B000808191819093FF0A8093FE0A87E797E7C2
:1038C000918380839BE088E10FB6F894A89580935C
:1038D00060000FBE9093600083CF6C960FB6F89493
:1038E000DEBF0FBECDBFDF91CF91FF91EF91BF91B2
:1038F000AF919F918F917F916F915F914F913F9188
:103900002F911F910F91FF90EF90DF90CF900F902C
:103910000FBE0F901F901895CF92DF92EF92FF92FB
:103920000F931F93CF93DF936C017A018B01C0E05B
:10393000D0E0CE15DF0589F0D8016D918D01D6015B
:10394000ED91FC910190F081E02DC6010995892B44
:1039500011F47E0102C02196ECCFC701DF91CF9117
:103960001F910F91FF90EF90DF90CF9008953FB798
:10397000F8948091BC059091BD05A091BE05B091D1
:10398000BF0526B5A89B05C02F3F19F00196A11DC4
:10399000B11D3FBFBA2FA92F982F8827820F911DE5
:1039A000A11DB11DBC01CD0142E0660F771F881F2C
:1039B000991F4A95D1F708950895089580E090E001
:1039C00008950E94FE308F929F92AF92BF92CF9245
:1039D000DF92EF92FF926B017C010E94B71C4B01BA
:1039E0005C01C114D104E104F104F1F00E94B71CA0
:1039F000DC01CB0188199909AA09BB09883E9340CB
:103A0000A105B10570F321E0C21AD108E108F1085F
:103A100088EE880E83E0981EA11CB11CC114D1044D
:103A2000E104F10419F7DDCFFF90EF90DF90CF9024
:103A3000BF90AF909F908F9008951F920F920FB6F6
:103A40000F9211242F933F938F939F93AF93BF9324
:103A500080919E0190919F01A091A001B091A10140
:103A60003091BB0523E0230F2D3720F40196A11DD3
:103A7000B11D05C026E8230F0296A11DB11D20939C
:103A8000BB0580939E0190939F01A093A001B093EA
:103A9000A1018091BC059091BD05A091BE05B0919A
:103AA000BF050196A11DB11D8093BC059093BD0576
:103AB000A093BE05B093BF05BF91AF919F918F9129
:103AC0003F912F910F900FBE0F901F9018954F921E
:103AD0005F927F928F929F92AF92BF92CF92DF922E
:103AE000EF92FF920F931F93CF93DF9300D000D0FC
:103AF000CDB7DEB729011C2DA02EB12C9C012A0DBB
:103B00003B1D121613060CF0B3C1803891050CF062
:103B1000AFC1FB01EE0DF11D1E161F060CF0A8C172
:103B2000603471050CF0A4C14115510509F4A0C120
:103B3000E62FE770FE2EFB0177FD3796A3E0F595A3
:103B4000E795AA95E1F7AE2F77FF04C0FF2011F0AB
:103B5000AFEFAE0F97FF05C0EE27FF27E81BF90B6D
:103B600002C0E0E0F0E02038310524F020E8722EB9
:103B7000781A01C0702E7E1A6A2F0A2E000C770B5D
:103B8000AF3F1CF4D62ED09401C0D12C21E03E2DA5
:103B9000377009F420E0E694E694E694E20E6E0DA8
:103BA000711D693071051CF028E0E22EEA1AED184B
:103BB0003D2D3A0FDC0120E83203A00DB11D112488
:103BC000AE0FBF1FD09EE00DF11D11244E0F5F1FE1
:103BD00081E090E04C010F2C02C0880C991C0A94E3
:103BE000E2F7133009F403C1A0F4113009F4B5C0B1
:103BF000123009F03DC18FEF889DB001899D700D95
:103C00001124609570957C836B835C802E2D230F2F
:103C10002BC01A3F31F01B3F09F02AC12E2D230F74
:103C200088C02E2D230F51C0FA01E00FF11FE4913F
:103C3000E89D6001E99DD00C1124DA82C98237FD2C
:103C400007C0FC01E080EE2DE623CE2AFC01C082F5
:103C5000F11013C00F5F1F4F0196071528F33F5F48
:103C60004A0D5B1DA058BF4F321709F401C1CD01A9
:103C70008C559E4F00E010E0F0CF37305CF7FC0130
:103C8000E058FF4FD080D520CA80DC28D082E2CF18
:103C9000FA01E60FF71FE491E89D8001E99D100D00
:103CA00011241A83098337FD04C0FC011081012B04
:103CB0000083F11013C06F5F7F4F0196671540F3CB
:103CC0003F5F4A0D5B1DA058BF4F321709F4D0C0AB
:103CD000CD018C559E4F60E070E0F0CF37305CF73F
:103CE0008C0100581F4FF801E080EA81EE2AF801AC
:103CF000E082E1CFFA01E00FF11FE491E89DC001FD
:103D0000E99D900D11249A83898337FD05C0809524
:103D1000FB01908189238083F11014C00F5F1F4F36
:103D20006F5F7F4F071530F33F5F4A0D5B1DA05853
:103D3000BF4F321709F49CC0BD016C557E4F00E0A7
:103D400010E0F0CF373054F7FB01E058FF4F8A8185
:103D50008095908189238083E1CFC2018E0F9F1FC0
:103D60002E2D230F321709F483C0BD016C557E4FF1
:103D70006B0100E010E0071590F5FC01E00FF11F6A
:103D8000E491E89DB001E99D700D11246095709556
:103D90007C836B83FA01E00FF11FE491E89D200121
:103DA000E99D500C11245A82498237FD05C0F60165
:103DB00070816723462A4082FF2059F037304CF447
:103DC000F601E058FF4F70816C8167237A81672B81
:103DD00060830F5F1F4FFFEFCF1ADF0ACCCF3F5F2B
:103DE0004A0D5B1D8A0D9B1DA058BF4FBBCFC72C32
:103DF000D12CE40FF51FAC55BE4F60E870E06C1994
:103E00007D09AC18BD088501000F111F572D2E2DFF
:103E1000CF93DF93ED01EF96EF962296A590C59094
:103E2000FF2059F0A89C5001C89C600137302CF449
:103E3000E880D094ED20EB28E99233233AF0EC901F
:103E4000C094EC20EA28ED920C94271F11965A9505
:103E500029F72A9551F0572D33951124E00FF11DC4
:103E6000A60FB11DC60FD11DD9CFDF91CF9111245F
:103E70000F900F900F900F90DF91CF911F910F91A6
:103E8000FF90EF90DF90CF90BF90AF909F908F907A
:103E90007F905F904F9008952D9A0895BC0180E027
:103EA00090E00C94E31C8FB18095807F669B8860C6
:103EB0001C9B846008951092A2013E983F9808953B
:103EC0003E9A3F9A81E08093A20108952F923F92FB
:103ED0004F925F926F927F928F929F92AF92BF921A
:103EE000CF92DF92EF92FF920F931F93CF93DF93C6
:103EF000CDB7DEB72D970FB6F894DEBF0FBECDBF9E
:103F0000ED82E22EF12C9C012E0D3F1D37FD32C1BA
:103F1000803891050CF02EC19B01200F311D37FD1B
:103F200029C1603471050CF025C1DB0177FF04C0A5
:103F3000AA27BB27A61BB70BA770BB279B0177FF40
:103F400002C0295F3F4F13E0359527951A95E1F799
:103F500077FF08C02150310968E070E0FB01EA1BDF
:103F6000FB0BDF01E02FE695E695E695CE2ED12CF2
:103F7000077019F0FFEFCF1ADF0AB9017695762F97
:103F8000662777956795680F791F6C557E4F860178
:103F9000020F131F19870887C12CD12CF8E0AF2E10
:103FA000B12C85010A1B1B0B1F830E830885198505
:103FB0002017310709F4DEC02830310509F4DAC0D2
:103FC0002F3F1FEF31070CF4CAC08B0100581F4F61
:103FD0001D870C874B013B012B011C011C830B83AC
:103FE0001A8309831B861A860A851B850E151F05F1
:103FF0000CF0B5C010E82116310409F4B0C037FC4C
:1040000089C02F3FEFEF3E0709F4B0C00A851B853A
:104010000C0D1D1DFD81F13079F4F801E40FF51F41
:10402000E491F0E08F010A2E01C0000F0A94EAF734
:10403000F301B0800B2925C0FD81F11114C0F801F6
:10404000E40FF51FE491F0E00A2E02C0EE0FFF1F0F
:104050000A94E2F78F0100951095F401A080B12C2D
:104060000A211B210EC0F801E40FF51FE491F0E0D6
:104070008F010A2E01C0000F0A94EAF7F201B08006
:104080000B250083109709F445C02730310509F44A
:1040900041C00A851B850C0D1D1DFD81F13089F481
:1040A000F801E40FF51FE4910E2F10E00E8002C01E
:1040B000159507950A94E2F7EC85FD85B0800B29EC
:1040C00028C0FD81F11115C0F801E40FF51FE4913E
:1040D0000E2F10E00E8002C0159507950A94E2F7A6
:1040E00000951095E981FA81A080B12C0A211B214D
:1040F00010C0F801E40FF51FE4910E2F10E00E80C0
:1041000002C0159507950A94E2F7EB81FC81B08017
:104110000B2500830A851B850F5F1F4F1B870A87AE
:104120000C851D850F5F1F4F1D870C8709811A8124
:104130000F5F1F4F1A8309830B811C810F5F1F4F75
:104140001C830B831FEF211A310AEFEF4E1A5E0A10
:10415000FFEF6F1A7F0A0FEF801A900A45CF2F5F8B
:104160003F4F60587F4FCE0CDF1C20CF109709F0D7
:1041700090CFD0CF2D960FB6F894DEBF0FBECDBF37
:10418000DF91CF911F910F91FF90EF90DF90CF9033
:10419000BF90AF909F908F907F906F905F904F9067
:1041A0003F902F90089560387105D0F44034510548
:1041B000B8F4E4E3F4E080E1849FD001A078112416
:1041C000A60F4770E40FF11D8491AC55BE4F22231A
:1041D00019F06C91862B03C080956C9186238C938B
:1041E00008952F923F924F925F926F927F928F929B
:1041F0009F92AF92BF92CF92DF92EF92FF920F9376
:104200001F93CF93DF93CDB7DEB729970FB6F894FE
:10421000DEBF0FBECDBFFC016A3069F425898189FC
:10422000928938E0239F800D911D1124928B818B00
:10423000108A1786AAC06D3009F4A7C099878887AD
:10424000F58834882388618872880785108900384A
:104250001105C4F0A885B98555962C915597422F24
:1042600050E01F968D919C915097B6E02B9F800D4A
:10427000911D1124E885F985908B87872689211166
:104280006EC083C0F0E46F16710424F7C80125E006
:10429000F29E800D911D112418161906DCF68F2D43
:1042A00090E09C838B83C301A8E0FA9E800D911D52
:1042B00011241816190674F6B5E06B9FB00111248D
:1042C000FB01E45CFB4FFA83E98330E08885998544
:1042D00004969E838D83E981FA81E490353009F458
:1042E000E12C430188E0482EE0FC02C0532C01C0C1
:1042F000522C51100BC0321009C0E6944A948B81A5
:104300009C81880E991E4110EFCF1BC068018C2D37
:10431000801B8F1590F754018A2D88198F1568F42A
:10432000252DA501B6018D819E813F830E94D3205A
:104330009FEFA91AB90A3F81EFCFAFEFCA1ADA0A85
:10434000E6CF3F5FEB81FC810E0F1F1F89819A81B1
:1043500001969A838983363009F0BDCF7BCF6AEF0F
:1043600064039001659F300D112420583F4F28179A
:1043700039075CF4A885B985ED91FC9111970190FE
:10438000F081E02D6AE0CD01099581E090E0299669
:104390000FB6F894DEBF0FBECDBFDF91CF911F9156
:1043A0000F91FF90EF90DF90CF90BF90AF909F90D4
:1043B0008F907F906F905F904F903F902F900895D7
:1043C0000F931F93CF93DF9300D000D01F92CDB7F0
:1043D000DEB749835A836B837C838D83F8016081C8
:1043E000718162337105B8F485E0869FA001879FD3
:1043F000500D1124D901A40FB51FFE013196019073
:104400000D928A95E1F7F80180819181019691835F
:10441000808381E001C080E00F900F900F900F909B
:104420000F90DF91CF911F910F9108952F923F929E
:104430004F925F926F927F928F929F92AF92BF92B4
:10444000CF92DF92EF92FF920F931F93CF93DF9360
:10445000CDB7DEB728970FB6F894DEBF0FBECDBF3D
:104460006E834F83322EE8862601282E82E3821542
:1044700010F482E3282EC02ED12CEE24FF24EC1859
:10448000FD08612C712C362D621408F042C0832F78
:1044900068850E94C430911108C0EC18FD08232DD6
:1044A000E3E0E31518F423E001C020E04E814B3037
:1044B00008F04AE06F816B3008F06AE070E0641B3E
:1044C00071096F5F7F4FC3010E94E430480FF20112
:1044D000668D832F0E94C4307E2DFD82EC82F0E435
:1044E0002F9F9001112484E0489FF0011124EF5682
:1044F000F74F51815F73522B4F70EC18FD08840108
:104500009501692F8D810E94E021EFEF6E1A7E0ADE
:10451000BACF28960FB6F894DEBF0FBECDBFDF919D
:10452000CF911F910F91FF90EF90DF90CF90BF90B0
:10453000AF909F908F907F906F905F904F903F9043
:104540002F900895CF93DF93CDB7DEB727970FB69F
:10455000F894DEBF0FBECDBF877097E0899FF00152
:104560001124EB5DFE4F87E0DE01119601900D9264
:104570008A95E1F729813A814B815C816D817E8149
:104580008F8190E027960FB6F894DEBF0FBECDBFA7
:10459000DF91CF91089582E08093A40580E4809319
:1045A000900087E597E09093990080939800089594
:1045B0001F93CF93DF931F92CDB7DEB7182F809153
:1045C000CA05812321F48091C905812341F5662321
:1045D00071F10E94531F8123811317C080910C0138
:1045E000811111C08091C7059091C80566E070E007
:1045F0000E94D030892BD9F4812F0F90DF91CF9179
:104600001F910C94F70F815010C08091CA0581232F
:1046100071F08091C905812351F484E106C0812F96
:1046200069830E94F70F6981D2CF80930C010F90AC
:10463000DF91CF911F9108952F923F924F925F92F9
:104640006F927F928F929F92AF92BF92CF92DF92A2
:10465000EF92FF920F931F93CF93DF93CDB7DEB707
:1046600027970FB6F894DEBF0FBECDBF8C01562E34
:10467000FC01108213823090880840908908C32C76
:10468000D12CF0E14F9E500111247501EC0CFD1C62
:104690004701880C991CC4018E0D9F1DFC01E95235
:1046A000FA4F26A4662E712C2EE0221212C0FC01B5
:1046B000EA5FF94F80810E94A22229833A834B83CB
:1046C0005C836D837E838F8345E0451508F098C138
:1046D00019C087E0E5E2F1E0DE01119601900D924C
:1046E0008A95E1F785E0861760F0E8E16E9FC001EA
:1046F00011248C58964FF80192838183211015C0A4
:1047000017C068E0C30173E0880F991F7A95E1F73D
:10471000845F964FF80192838183F7E0F51508F4E2
:1047200005C1211002C0311034C181E0F80180833D
:1047300087E0869DF001879DF00D1124EB5DFE4F13
:104740008481F8018383F9E05F120BC0F401EE0D60
:10475000FF1DEA5FF94F808187708650823008F430
:1047600014C1F801838190E020918308309184087E
:104770002817390730F480910306813011F081E069
:104780008083852D90E08D30910508F0CCC0FC0130
:10479000E35AFF4F0C94F83087E6F801848385E7ED
:1047A000858381E6868382E7878384E635C083E656
:1047B000F801848381E685838EE6868387839FE67E
:1047C000908712C089E6F801848383E6858385E6B5
:1047D0009CC085E6F80184839CE69583868383E606
:1047E000878384E7808782E78187128613C183E706
:1047F000F80184838EE6858389E6868380E7878354
:1048000085E6F0CF8DE6F801848381E6858387E62F
:10481000868389E6878383E680871186FBC087E7E6
:10482000F801848381E6858384E7868385E6878330
:1048300082E7F2CF86E6F801848389E6858382E702
:10484000868385E66DC0F401EE0DFF1DE952FA4F37
:1048500086A58E3009F067C081E090E0F8E05F1235
:1048600002C080E090E0FE01E80FF91F86819BE224
:10487000F8019483823049F160F4882309F1813092
:1048800009F051C083E7F801858380E7868384E6D9
:1048900047C0833009F1843009F045C083E7F8014F
:1048A000848380E7858384E6868380E2878381E64C
:1048B000808795E7918792E7928783871486AAC0BD
:1048C00084E6F80185838DE604C082E7F8018583DC
:1048D0008EE6868387E624C083E7F801848388E632
:1048E00085838FE6868383E687838BE695CF83E790
:1048F000F801848385E685838CE6868311C087E68C
:10490000F80184838FE6858381E28683178282C0E3
:1049100081E7F801848385E7858389E6868384E7D8
:104920008783108677C0F801148274C0F9E0F5150A
:1049300028F1F401EE0DFF1DEA5FF94F208130E010
:10494000F8E05F1619F080E490E002C080E890E0A3
:1049500028233923232B21F081E0F8018083F3CE33
:10496000FEE02F12F9CF862F90E0880F991F63E0A9
:1049700070E00E94E430F8016383E5CEFAE05F1254
:10498000E2CE2EE0221609F4ECCE81E0F80180831D
:10499000E8CE442009F4C9CE3A94232D30E0A20E8B
:1049A000B31EF501EE0FFF1FCF018A0D9B1DFC0109
:1049B000E952FA4F86A58111B8CE4A94F0E14F9E94
:1049C000C0011124C80ED91EF601EE0FFF1FAF0162
:1049D0004C0D5D1DFA01E952FA4F46A54111A5CED5
:1049E000820F931FFC01EE0FFF1F8E0F9F1FFC0114
:1049F000E952FA4F81E096A5911198CE80E096CECB
:104A0000F8E15F9EC00111248C58964FF801928303
:104A100081838BCEC80127960FB6F894DEBF0FBEF8
:104A2000CDBFDF91CF911F910F91FF90EF90DF905D
:104A3000CF90BF90AF909F908F907F906F905F903E
:104A40004F903F902F9008950F931F93CF93DF9334
:104A50008C01C0E0D0E0F801EC0FFD1F64916623EB
:104A600071F0E091C005F091C1050190F081E02D59
:104A700080EC95E00995892B11F02196ECCFCE01C1
:104A8000DF91CF911F910F910895009769F0FC017C
:104A900001900020E9F73197AF01481B590BBC0189
:104AA00080EC95E00C948C1C80E090E008958F924F
:104AB0009F92AF92BF920F931F93CF93DF93CDB787
:104AC000DEB7A1970FB6F894DEBF0FBECDBF19A217
:104AD000423008F44AE08E010F5D1F4F842E912C66
:104AE000A12CB12CA50194010E949330E62FB901AD
:104AF000CA0101501109EA3014F4E05D01C0E95C1B
:104B0000D801EC93232B242B252B61F7C8010E949D
:104B10004525A1960FB6F894DEBF0FBECDBFDF913D
:104B2000CF911F910F91BF90AF909F908F9008955C
:104B3000DF92EF92FF920F931F93CF93DF937C014D
:104B4000D22E8B01040F111DEB0177FF0EC0C0E0C8
:104B5000D0E00BC0C417D5077CF42D2DAE01B701F2
:104B600084EC95E00E94D3202196A8010134110520
:104B70008CF340E450E0EECFDF91CF911F910F9185
:104B8000FF90EF90DF900895CF92DF92EF92FF9227
:104B90000F931F93CF93DF936B01122FEC017C01D6
:104BA000E40EF11CCE15DF0544F4202F412FB60191
:104BB000CE010E9498252196F5CFDF91CF911F91CC
:104BC0000F91FF90EF90DF90CF900895AF92BF923A
:104BD000CF92DF92EF92FF920F931F93CF93DF93C9
:104BE000CDB7DEB72F970FB6F894DEBF0FBECDBF9F
:104BF000A982BA82CB82DC82ED82FE820F83188783
:104C000029873A874B875C876D877E878F8780915E
:104C1000F605823078F49FE0989FD0011124FE01C0
:104C20003196A852BA4F01900D929A95E1F78F5F95
:104C30008093F6052F960FB6F894DEBF0FBECDBF5A
:104C4000DF91CF911F910F91FF90EF90DF90CF9068
:104C5000BF90AF9008954091A7055091A80520916D
:104C6000A5053091A60542175307B4F49091E800CA
:104C70009570E1F39091E80092FD19C08093F100E6
:104C80008091A7059091A80501968F739927892B8C
:104C900019F48EEF8093E8008091A7059091A80504
:104CA00001969093A8058093A70581E0089580E080
:104CB0000895615030F02091F100FC0120830196AD
:104CC000F8CF289884E68093AC050895CF93DF93BE
:104CD000CDB7DEB7E5970FB6F894DEBF0FBECDBFF8
:104CE000789484B5826084BD84B5816084BD85B5C7
:104CF000826085BD85B5816085BD80916E008160D3
:104D000080936E0010928100809181008260809378
:104D1000810080918100816080938100809180007A
:104D200081608093800080919100826080939100E7
:104D300080919100816080939100809190008160CA
:104D4000809390008091C10084608093C100809125
:104D5000C10082608093C1008091C1008160809316
:104D6000C1008091C30081608093C3008091C00026
:104D700082608093C0008091C20081608093C200F5
:104D800080917A00846080937A0080917A008260BA
:104D900080937A0080917A00816080937A0080917C
:104DA0007A00806880937A001092AD051092AA056F
:104DB0001092AB058091D70081608093D70080EA84
:104DC0008093D80089B5806189BD89B5826089BD2D
:104DD00009B400FEFDCF61E070E080E090E00E9449
:104DE000E31C8091D8008F7C80618093D8008091F3
:104DF000E000807F8093E0008091E1008E7E8093D0
:104E0000E1008DE08093E200559A209AEEEFFFE7F3
:104E1000859194918B3F9C4D19F481E08093A90575
:104E200081EC80937C0085B1806F85B984B1877EE9
:104E300084B984B1876E84B95E9A5F988AB1806DB7
:104E40008AB9769A6E9881B3806F81BB899880B356
:104E50008D7080BB80E58CBD81E08DBD85E090E0EC
:104E60000E944E1F5F9A85E090E00E944E1F5E9860
:104E70005C98E4E8F1E08DE08E0F94919EBD000017
:104E80000DB407FEFDCF31968E13F7CF5C9A81E803
:104E9000809364008091650081608093650080E06C
:104EA0000E9427160E94531F87FF15C05C9885EA51
:104EB0008EBD00000DB407FEFDCF5C9A2E982F9892
:104EC0002D988091640080628093640081E083BFAC
:104ED000889513BEFCCF02E010E00E94531F82FFB2
:104EE00042C02D980E94531F84788438C9F00E94D4
:104EF000531F8471843191F50E944C1F88EC90E01F
:104F00000E944E1F2E981A83098360E0CE010196FD
:104F10000E94D70F84EF91E00E944E1F2E9A19C075
:104F20000E944C1F88EC90E00E944E1F2F981A831D
:104F300009836FEFCE0101960E94D70F84EF91E0B5
:104F40000E944E1F2F9A0E94531F84788438D9F3F1
:104F5000CECF0E94531F84718431D9F388EC90E046
:104F60000E944E1FBACF0E944C1F82E090E00E9428
:104F70004B30882319F00E94601F02C00E945B1F03
:104F800081E090E00E944B3082FB112710F981E014
:104F900090E00E944B3081FF46C011112E9850EFD7
:104FA000C52EDD24DA940E94531F86FF04C02E9A7A
:104FB0002F9A2D9A38C0112331F034E0C316D10452
:104FC00011F42E9A2F9881E00E942716EE24E39484
:104FD00000E128E544ED50E0B60184E190E00E9454
:104FE000661F80E00E9427168FE090E00E944E1F0F
:104FF0004FEFC41AD40A59E1C516D104A1F6112302
:1050000011F02F9A2D9880E991E00E944E1F0E9486
:105010004C1FE091C405F091C5050190F081E02D91
:1050200084EC95E0099582E390E00E944E1F0E9477
:10503000531F8111F8CF8091A20180938B081092A9
:1050400090008AE0809391000E94141680E1809382
:10505000CB058AEC90E00E944B300BEC10E08F35D2
:1050600069F4C8010E944B30F801EF53F84F808378
:105070000F5F1F4F003D1105A1F715C01A8309836B
:1050800060E0CE0101960E94D70F0F5F1F4F003DD9
:105090001105A1F78AEC90E09A8389836FE5CE0130
:1050A00001960E94D70F8FB7F89440919E015091BE
:1050B0009F016091A0017091A1018FBF8091CC05EB
:1050C000942F981B892F9091CD05992329F08093D7
:1050D000CE051092CD05BDC49091CB05891748F43B
:1050E0008F5F891708F0B5C481E083BF889513BE30
:1050F000B0C481E08093CD054093CC058091C70575
:105100009091C80501969093C8058093C70580913A
:10511000A405882331F081508093A405882309F4E5
:10512000A0C48091C9058093CA050E94531F809333
:10513000C90560E088E00E94D82260E084E00E9417
:10514000D82261E080E20E94D82261E080E40E94DF
:10515000D82261E080E80E94D82261E080E10E94CC
:10516000D8220E94531F87FF04C00E94531F82FD54
:105170007BC48091D705833019F0A1E0AEA70DC0A4
:105180000E94531F83FFF9CF0E94531F82FD03C06B
:10519000B1E0BEA702C0E5E0EEA71DA680918108A0
:1051A0009091820801969093820880938108809163
:1051B000D705833009F0A0C2E12CA5E0FA2EB3E0B8
:1051C000CB2ED12C15E0912E00E4802E8CE1A82E60
:1051D00085E1B82E2E2D30E080917F0890918008D7
:1051E0002817390708F0C1C0F29E8001F39E100D08
:1051F00011240B57184FE0918108F0918208D801D3
:1052000011968C9111978F73C9F06C91A62FAF7086
:1052100044E0A49FD0011124AF56B74F12968C9151
:1052200062956F7009F06FE0680F70E0660F771F8E
:10523000CF010E94D030892B09F41EC4CF01B601E2
:105240000E94D030892B79F4D8014C91842F82951B
:105250008F7049F08150B0E18B9FC00111244F70D5
:10526000842BF8018083D80111968C918F7311F1F2
:10527000F29EF001F39EF00D1124E952FA4FDF0186
:10528000A055BE4FAC91EF54FE4F2FE0A29FD0012E
:105290001124A852BA4F13968D919C91149733E024
:1052A000880F991F3A95E1F7208131812817390736
:1052B00094F52FC0D8018C918F70863051F5F29EF5
:1052C000F001F39EF00D1124E952FA4FDF01A055D1
:1052D000BE4FAC91EF54FE4F2FE0A29FD00111249E
:1052E000A852BA4F13968D919C91149723E0880F82
:1052F000991F2A95E1F720813181281739074CF44D
:10530000CCC39092A40580929000B0929900A09294
:105310009800E3945FCFC8010E942A078091850816
:1053200090918608D801EC91EF70B4E0EB9FF0010A
:105330001124EF56F74F2381821B910997FDAAC3D1
:105340009093860880938508892BD9F685E0809311
:10535000D7058FE08093A40580E48093900082E8D5
:1053600093E29093990080939800809185089091A2
:105370008608892B09F4C0C1E6E0F6E0FAA7E9A7A0
:10538000412C512CE42C442021F04FEF440D4FA729
:1053900001C01FA656E04516510424F481E08E0D8D
:1053A00088AB02C097E098AB29A43AA4AFEF2A1AC1
:1053B0003A0A09A51AA5F12CF101329780818E30A5
:1053C00051F0F3940D5F1F4FF3E02F0E311C20E1DD
:1053D000F212F2CF3FC1C0908108D0908208309184
:1053E0007F083BA7D8018C910E94A22229833A838F
:1053F0004B835C836D837E838F836F2D7E2DCE01E7
:1054000001960E9416074C01C8010E94D106B82ED1
:10541000D101EC91EF3F09F04CC0E5E86E2EE7E0DA
:105420007E2ED12CF5E0CF2EFBA5DF1608F074C040
:10543000F301DE0111968C2D01900D928A95E1F712
:105440008C819D8197FD30C08A818F7369F169815C
:105450006F70C8010E94FB06882331F168ED75E08A
:10546000CE0101960E9412084B2DB4010E947E0FBE
:1054700081111AC0F101D082D8018C91877C8C9364
:105480000E94CB22F80180818770823009F044C0ED
:10549000D101EC91B5E0EB9FF0011124EB57F84FEF
:1054A000808182958F70C1F1D394E5E06E0E711CFE
:1054B000BBCF25E0E29FF0011124EB57F84F85E0C8
:1054C000DE01119601900D928A95E1F78A818F7322
:1054D00009F431C38C819D8197FD2DC3F801B08003
:1054E0008B2D0E94A2222AA33BA34CA35DA36EA3F3
:1054F0007FA388A761E0C8014DAB0E94A5064DA916
:1055000081111DC380E0481B642F70E0C6010E941A
:10551000D030892B09F415C38091810890918208BD
:1055200087709927892B09F04CCF64E0C8010E944D
:10553000A506882309F445CFFF2039F0AA24AA94B0
:10554000AF0CFDE0FF1530F001C0A12CBB24B394DB
:10555000BF0C02C07FE0B72ECFA4662463946B0C0F
:10556000712C48A94C1508F42CCF50E1C59E400180
:105570001124C401860D971D9C01220F331F820F39
:10558000931F9C0129523A4FD9019E96BCA7ABA705
:10559000FC01EA5FF94FFAABE9ABDA2C3CAB2BAB81
:1055A000BD1408F455C0DF1003C0CE1409F44EC07A
:1055B000C4018D0D911D9C01220F331F820F931F7B
:1055C000FC01E952FA4F26A52E3049F4BE96DC01C3
:1055D000AA5FB94F8C918770853009F537C0DB1011
:1055E00035C02EE02D1590F1ABA9BCA99E968C91EB
:1055F0008E3061F5E9A9FAA980810E94A22229834F
:105600003A834B835C836D837E838F83265081E056
:10561000223008F080E0EBA5FCA58823B9F02181B9
:10562000922F9873892F90E053E0959587955A951E
:10563000E1F78630910514F48E5F01C087E038E011
:10564000839FC0011124277C822B8183D394A8CF10
:10565000C39487CFFFEF4F1A5F0A29A53AA5205DB3
:105660003F4F3AA729A738E04316510409F08ACEE4
:1056700040917F085091800880E065E0282F30E05D
:105680002417350760F4629FF001639FF00D112429
:10569000EB57F84F91819F7379F58F5FEFCF209192
:1056A000870880918308909184080596322F36955B
:1056B0003695830F911D90938408809383082F5F04
:1056C0002093870882E08093D70547ED55E028E0D6
:1056D0003FEF80E090E0FA01E80FF91F30AB03964E
:1056E00080339105C1F72150405D5F4F2111F1CF0B
:1056F0001092800810927F08BDA5BF5FBDA7EEA5E0
:10570000BE134CCD0E9414168091D70581110EC195
:1057100001E020E440E860E070E080E090E00E947A
:10572000C42500E022E149E165E070E083E390E018
:105730000E94C425EE24E39402E129E141ED51E009
:1057400065E070E083E390E00E94661F40E065E062
:1057500070E089E190E00E944B1842E065E070E063
:1057600086E590E00E944B1800E025E040E86CE1FF
:1057700070E080E090E00E94C425C12CD12C9FE015
:10578000A92EB12C8091810890918208B5010E94C8
:10579000D030EE24E39405E02FE042EC51E06CE1E0
:1057A00070E0D601A81BB90BCD010E94661FBFE0B7
:1057B000CB0ED11CE6E9CE16D10421F7E0918A0880
:1057C0001A821A8A1982E53090F580E28A838B83E7
:1057D0009DE69C8391E69D8390E79E838F8391E372
:1057E0009E0F988789878A871B8692E69A8B95E613
:1057F0009B8B93E79C8B94E79D8B9AE39E8B8F8B7F
:10580000F0E0E457F74F80811F928F938BE991E08E
:105810009F938F93CE0148969F938F930E9403315D
:105820000F900F900F900F900F900F9021C0E530C8
:10583000E9F480E28A8393E79B839EE69C8394E667
:105840009D839AE39E838F838FE6888780918B0860
:10585000811102C096E601C09EE69987811102C0BF
:1058600086E601C080E28A871B8602C082E08983C7
:1058700000E02BE040E866E270E080E090E00E940B
:10588000C42511E01093D3051092D40586E190E071
:105890009093D0058093CF0588E290E09093D20555
:1058A0008093D1056CE380EC95E00E94F12060E2EA
:1058B00080EC95E00E94F120CE0102960E944525E1
:1058C00060E280EC95E00E94F1206EE380EC95E0D0
:1058D0000E94F1201092D3051093D40582E090E04D
:1058E0009093D0058093CF0587E390E09093D20505
:1058F0008093D105CE0142960E94452580910306F2
:10590000882309F454C08091810882FD50C08FE241
:1059100090E09093D0058093CF058AE190E090933A
:10592000D2058093D1058BEB91E03CC08530E9F541
:1059300001E020E440E860E070E080E090E00E9458
:10594000C4251092D30581E08093D40504E110E0D2
:105950001093D0050093CF058AE090E09093D20594
:105960008093D1058DEA91E00E94242560918708FB
:1059700070E080E090E04AE00E945725E091040644
:10598000F0E0E457F74F909187088081891778F409
:105990001093D0050093CF051093D2050093D10545
:1059A00081EA91E00E94242502C00E949208809121
:1059B000D705843031F501E02CE24CE66AE070E076
:1059C0008AE090E00E94C4252CE24CE66AE070E098
:1059D0008AE090E00E941B181092D30581E080932A
:1059E000D40582E190E09093D0058093CF058CE1BF
:1059F00090E09093D2058093D10581E991E00E94D7
:105A000024258091D705853081F4609187088091A5
:105A1000040690E0FC01E457F74F2081261738F484
:105A20002091A301211103C01EC11092A3018091F6
:105A30008B089091A201981749F0882319F00E94D1
:105A4000601F02C00E945B1F0E94CB2280E00E9468
:105A5000271680E090E0892B09F425CB0E940000F6
:105A600022CB109290005DCB0E94531F91E084FFE7
:105A700090E0909303067DCBF29ED001F39EB00D93
:105A80001124A857B84F8D919C91119701968D9331
:105A90009C93D4CB80E090E053CCF80143815481B7
:105AA000B281A0919208AF731082A1834A5051092C
:105AB00020917F08309180082233310598F4F29EBE
:105AC000F001F39EF00D1124EB57F84F1082A183E3
:105AD000B283548343832F5F3F4F309380082093DA
:105AE0007F0817CC712C612C672D70E0621773074B
:105AF000A0F4F69EC001F79E900D1124FC01EB5717
:105B0000F84F81818F7339F41082A183B28354835B
:105B10004383662463947394E7CF6110FACBD80172
:105B200011968C91119782958695869583708064E5
:105B300011968C93EECB8FEFD1018C93EDCC82E05C
:105B4000E2CC8B2D88738695869586958F5F8770BE
:105B500038E0839FC0011124D8019C91977C892B48
:105B60008C93887309F0D8CCF1016081F5E06F9FC8
:105B7000B00111246B57784F20E043E858E0C8018A
:105B80000E945F07D8018C918770813011F18730B6
:105B900001F1823019F48FEFD1018C93F1018081F2
:105BA0008F3F09F4B9CC68ED75E0CE0101960E94F3
:105BB00012086C01C8010E94D106482FB401C60129
:105BC0000E947E0F811148C08C819D8197FF48C043
:105BD00043C0D1018C91B5E08B9FC001112468EDC9
:105BE00075E08B57984F0E9412083C0186E8C82E3A
:105BF00087E0D82E30E0EBA53E1780F6F1018081DA
:105C00003817D9F05601F1E0AF1AB108D6018C91DE
:105C10008F7399F012968D919C91139797FD0DC0FB
:105C200068ED75E0C5013DAB0E9412084CE0B30180
:105C30000E947E0F3DA9882329F03F5FB5E0CB0E7F
:105C4000D11CD9CF21E043E858E0B501C8013DABF4
:105C50000E945F073DA9F1CF8FEFF10180835CCCFB
:105C60000E94CB2259CC85539F4F9A838983CE01C2
:105C700001960E94D70F81E08093A301D8CECF92E6
:105C8000DF92EF92FF920F931F93CF93DF931F92B8
:105C9000CDB7DEB7182F062FE42E862F880F8E5F24
:105CA00099830E942B2683E00E942B26F12EC12E81
:105CB0009981D92E8C2D8F19801798F4F601E7FE63
:105CC00002C0849101C080810E942B26182F80E0A1
:105CD0000E942B268123FFEFCF1ADF0A8111EACF22
:105CE00001C081E00F90DF91CF911F910F91FF9044
:105CF000EF90DF90CF9008950F931F93CF93DF9392
:105D00008C0181E090E00E944B3080FF32C08AE03D
:105D100090E00E944B309FEF980F9E3F50F522E39A
:105D200030E0D80150963C932E931F9728E330E043
:105D300052963C932E935197CBE0D0E0D801ED9151
:105D4000FC910190F081E02D682FC8010995CE01EA
:105D50000E944B302196C131D10581F780E00E942D
:105D6000271688EE93E0DF91CF911F910F910C944D
:105D70004E1FDF91CF911F910F91089504970C94BE
:105D80007C2ECF93DF931092C0081092BF0888EE4C
:105D900093E0A0E0B0E08093C1089093C208A09384
:105DA000C308B093C40881E691E09093BE08809345
:105DB000BD088FEF9FEF9093CA088093C908109297
:105DC000910847E04093920892E09093930881E015
:105DD000809394088093950838E0309396088093D8
:105DE000970880939808909399082CE020939A083C
:105DF00090939B0880939C0823E020939D08C4E126
:105E0000C0939E0890939F088093A00854E05093FD
:105E1000A1086DE06093A2088093A3088093A40872
:105E200065E06093A5086BE26093A6085093A7080D
:105E30009093A80856E05093A908C093AA0890939D
:105E4000AB089093AC084093AD084EE14093AE0888
:105E50002093AF089093B0083093B1083AE33093A1
:105E6000B2089093B3082093B40899E09093B508D2
:105E70009FE39093B6088093B7082093B808DAE0C0
:105E8000D093B9089093BA088093BB082093BC08BC
:105E900088ED95E00E946D0F87EE95E00E946D0FF2
:105EA0001092F6051092F8051092F705C093F905C7
:105EB000D093FA0589E991E09093FC058093FB0566
:105EC00083E991E09093FE058093FD058DE891E0D4
:105ED000909300068093FF0587E891E09093020677
:105EE0008093010680E090E02FEFFC01E952FA4F29
:105EF00016A617A620AB0396803831E09307A9F7C2
:105F000080E090E02FEFFC01E952FA4F16A617A6A9
:105F100020AB0396803831E09307A9F7E7E8F7E074
:105F200087E4108212821182DF0111978C931197FE
:105F30001C92359698E0E138F90799F71092880895
:105F4000109289081092D705109282081092810849
:105F50001092800810927F0810928A08109203060F
:105F600010928B0810928C0810928D0810928E0857
:105F700010928F0810929008109204061092C30598
:105F80001092C2051092C9051092CA0580E1809353
:105F9000CB051092C8051092C7051092CD0583E776
:105FA00091E09093C1058093C00581E891E09093C2
:105FB000C5058093C4051092D0051092CF051092AC
:105FC000D2051092D10581E08093D3051092D405BB
:105FD0008093D5051092D605DF91CF9108958F92C9
:105FE0009F92AF92BF92CF92DF92EF92FF92CF93A8
:105FF000DF93EC01688179818A819B81611571054C
:106000008105910521F464E279ED8BE597E02DE1BE
:1060100033EF41E050E00E94613049015A019B0199
:10602000AC01A7EAB1E40E9480306B017C01ACEEC8
:10603000B4EFA50194010E948E30DC01CB018C0DE0
:106040009D1DAE1DBF1DB7FF03C00197A109B0483C
:1060500088839983AA83BB839F77DF91CF91FF9039
:10606000EF90DF90CF90BF90AF909F908F9008956A
:106070000E94EF2F08958DE091E00E94EF2F089588
:10608000A0E0B0E080930D0190930E01A0930F016A
:10609000B09310010895F999FECF92BD81BDF89A91
:1060A000992780B50895262FF999FECF1FBA92BD82
:1060B00081BD20BD0FB6F894FA9AF99A0FBE0196E9
:1060C0000895052E97FB1EF400940E94783057FD2A
:1060D00007D00E94933007FC03D04EF40C94783024
:1060E00050954095309521953F4F4F4F5F4F089504
:1060F00090958095709561957F4F8F4F9F4F089534
:106100000E94B530A59F900DB49F900DA49F800D67
:10611000911D11240895B7FF0C9480300E948030A7
:10612000821B930B0895A1E21A2EAA1BBB1BFD0133
:106130000DC0AA1FBB1FEE1FFF1FA217B307E40766
:10614000F50720F0A21BB30BE40BF50B661F771FBE
:10615000881F991F1A9469F760957095809590959E
:106160009B01AC01BD01CF010895A29FB001B39F77
:10617000C001A39F700D811D1124911DB29F700D50
:10618000811D1124911D0895991B79E004C0991F68
:10619000961708F0961B881F7A95C9F78095089581
:1061A000AA1BBB1B51E107C0AA1FBB1FA617B7073D
:1061B00010F0A61BB70B881F991F5A95A9F7809559
:1061C0009095BC01CD01089597FB072E16F400941D
:1061D00007D077FD09D00E94D03007FC05D03EF4EF
:1061E000909581959F4F0895709561957F4F089583
:1061F000EE0FFF1F0590F491E02D099481E090E0EF
:10620000F8940C94DB33AEE0B0E0E9E0F1E30C94F9
:10621000B2330D891E8986E08C831A8309838FEF40
:106220009FE79E838D83AE01475E5F4F6F89788DB8
:10623000CE0101960E9426312F813885F801E20FA8
:10624000F31F10822E96E4E00C94CE33ACE0B0E065
:10625000ECE2F1E30C94A4337C016B018A01FC01B4
:1062600017821682838181FFBDC1CE0101964C0148
:10627000F7019381F60193FD859193FF81916F0161
:10628000882309F4ABC1853239F493FD859193FFDE
:1062900081916F01853229F4B70190E00E940E339D
:1062A000E7CF512C312C20E02032A0F48B3269F062
:1062B00030F4803259F0833269F420612CC08D3281
:1062C00039F0803339F4216026C02260246023C075
:1062D000286021C027FD27C030ED380F3A3078F410
:1062E00026FF06C0FAE05F9E300D1124532E13C026
:1062F0008AE0389E300D1124332E20620CC08E327D
:1063000021F426FD6BC1206406C08C3611F4206890
:1063100002C0883641F4F60193FD859193FF819187
:106320006F018111C1CF982F9F7D9554933028F430
:106330000C5F1F4FFFE3F9830DC0833631F08337C5
:1063400071F0833509F05BC022C0F8018081898338
:106350000E5F1F4F44244394512C540115C0380143
:10636000F2E06F0E711CF801A080B18026FF03C01F
:10637000652D70E002C06FEF7FEFC5012C870E9492
:1063800003332C0183012C852F77222E17C038016F
:10639000F2E06F0E711CF801A080B18026FF03C0EF
:1063A000652D70E002C06FEF7FEFC5012C870E9462
:1063B000F8322C012C852068222E830123FC1BC07F
:1063C000832D90E048165906B0F4B70180E290E0C2
:1063D0000E940E333A94F4CFF50127FC859127FEF5
:1063E00081915F01B70190E00E940E3331103A9421
:1063F000F1E04F1A51084114510471F7E5C0843699
:1064000011F0893639F5F80127FF07C060817181E5
:10641000828193810C5F1F4F08C060817181072EBC
:10642000000C880B990B0E5F1F4F2F76722E97FF73
:1064300009C090958095709561957F4F8F4F9F4FC4
:106440002068722E2AE030E0A4010E944633A82E74
:10645000A81844C0853729F42F7EB22E2AE030E0F8
:1064600025C0F22FF97FBF2E8F36C1F018F4883582
:1064700079F0B4C0803719F0883721F0AFC02F2FE2
:106480002061B22EB4FE0DC08B2D8460B82E09C0E1
:1064900024FF0AC09F2F9660B92E06C028E030E086
:1064A00005C020E130E002C020E132E0F801B7FE93
:1064B00007C060817181828193810C5F1F4F06C08C
:1064C0006081718180E090E00E5F1F4FA4010E9407
:1064D0004633A82EA818FB2DFF777F2E76FE0BC023
:1064E000372D3E7FA51450F474FE0AC072FC08C01C
:1064F000372D3E7E05C0BA2C372D03C0BA2C01C003
:10650000B52C34FF0DC0FE01EA0DF11D80818033F2
:1065100011F4397E09C032FF06C0B394B39404C0AD
:10652000832F867809F0B39433FD13C030FF06C083
:106530005A2CB31418F4530C5B18B32CB31468F42E
:10654000B70180E290E03C870E940E33B3943C8513
:10655000F5CFB31410F43B1801C0312C34FF12C036
:10656000B70180E390E03C870E940E333C8532FF08
:1065700017C031FD03C088E790E002C088E590E0D5
:10658000B7010CC0832F867859F031FF02C08BE22F
:1065900001C080E237FD8DE2B70190E00E940E332A
:1065A000A51438F4B70180E390E00E940E335A94AA
:1065B000F7CFAA94F401EA0DF11D8081B70190E0B4
:1065C0000E940E33A110F5CF332009F451CEB7014C
:1065D00080E290E00E940E333A94F6CFF701868174
:1065E000978102C08FEF9FEF2C96E2E10C94C033AD
:1065F000FC010590615070400110D8F7809590958E
:106600008E0F9F1F0895FC01615070400190011092
:10661000D8F7809590958E0F9F1F08950F931F9325
:10662000CF93DF93FB01238121FD03C08FEF9FEF09
:1066300028C022FF16C04681578124813581421728
:10664000530744F4A081B1819D012F5F3F4F3183F7
:1066500020838C93268137812F5F3F4F378326839A
:1066600010C0EB01092F182F0084F185E02D09954A
:10667000892BE1F68E819F8101969F838E83812FE6
:10668000902FDF91CF911F910F910895FA01AA27C2
:10669000283051F1203181F1E8946F936E7F6E5F65
:1066A0007F4F8F4F9F4FAF4FB1E03ED0B4E03CD013
:1066B000670F781F891F9A1FA11D680F791F8A1FF6
:1066C000911DA11D6A0F711D811D911DA11D20D05D
:1066D00009F468943F912AE0269F11243019305D17
:1066E0003193DEF6CF010895462F4770405D419308
:1066F000B3E00FD0C9F7F6CF462F4F70405D4A3355
:1067000018F0495D31FD4052419302D0A9F7EACF1C
:10671000B4E0A6959795879577956795BA95C9F74B
:1067200000976105710508959B01AC010A2E06943E
:106730005795479537952795BA95C9F7620F731FF7
:10674000841F951FA01D08952F923F924F925F9234
:106750006F927F928F929F92AF92BF92CF92DF9271
:10676000EF92FF920F931F93CF93DF93CDB7DEB7D6
:10677000CA1BDB0B0FB6F894DEBF0FBECDBF09946A
:106780002A88398848885F846E847D848C849B84C1
:10679000AA84B984C884DF80EE80FD800C811B81CF
:1067A000AA81B981CE0FD11D0FB6F894DEBF0FBEFE
:0A67B000CDBFED010895F894FFCF6E
:1067BA00FFFFFFFF00E100000000000014010000DD
:1067CA0000080004060A0007030B050C090D00C1A6
:1067DA008081000000001E0602080201011B080257
:1067EA00080200021A0700110102032308041E000E
:1067FA0003043C05032D0102051908023C000406A6
:10680A002804076402010726060864020000000043
:10681A000085160617A6169B16EC16AA16C81600A9
:10682A00000000F1208C1CDE1CDD1C7C2EFCFF000D
:10683A0000BE2E000000002D0500000000670500C4
:0E684A00000000D005000000009B0525640042
:00000001FF
